:020000040800F2
:10000000980C0020ED010008894C0008BD40000854
:10001000F94B0008C10A0008A557000800000000BD
:100020000000000000000000000000000D4D00086E
:10003000F50A000800000000094D0008914D000875
:10004000070200080702000807020008070200086C
:10005000070200080702000807020008070200085C
:10006000070200080702000807020008C50A000886
:10007000D10A0008DD0A0008E90A000807020008A2
:10008000070200080702000807020008070200082C
:10009000070200080702000807020008070200081C
:1000A000070200080702000807020008070200080C
:1000B00007020008070200080702000807020008FC
:1000C00007020008070200080702000807020008EC
:1000D00007020008070200080702000807020008DC
:1000E000F90A0008070200080702000807020008D2
:1000F00007020008070200080702000807020008BC
:1001000007020008070200080702000807020008AB
:10011000070200080702000807020008070200089B
:10012000070200080702000807020008070200088B
:10013000070200080702000807020008070200087B
:10014000070200080702000807020008070200086B
:10015000070200080702000807020008070200085B
:10016000070200080702000807020008070200084B
:10017000070200080702000807020008070200083B
:10018000070200080702000807020008070200082B
:10019000070200080000000007020008070200082C
:1001A000070200080702000807020008070200080B
:1001B00007020008070200080702000807020008FB
:1001C00007020008070200080702000807020008EB
:1001D0000702000807020008DFF80CD000F01AFB45
:1001E00000480047A9570008980C0020064880479F
:1001F00006480047FEE7FEE7FEE7FEE7FEE7FEE70C
:10020000FEE7FEE7FEE7FEE7954D0008D90100088E
:100210002DE9F05F0546002092469B46884606463B
:10022000814640241BE0284641464746224600F0CE
:10023000F8F953465A46C01A914110D31146184650
:10024000224600F0DFF92D1A67EB01084F462246DF
:100250000120002100F0D6F917EB00094E41201EC5
:10026000A4F10104DFDC484631462A464346BDE896
:10027000F09FD2B201E000F8012B491EFBD270477B
:100280000022F6E710B513460A4604461946FFF762
:10029000F0FF204610BD2DE9FE4F804681EA0300A5
:1002A000C00F0C46009021F0004123F00045B8EB50
:1002B0000200A94105D24046214690461C460B4605
:1002C000024623F00040104347D0270DC7F30A0031
:1002D000C3F30A510290401A019040286BDAC3F32D
:1002E000130040F4801B0098924620B10023D2EB0B
:1002F000030A63EB0B0B01985946C0F140025046CC
:1003000000F080F906460D4650465946019A00F025
:1003100098F910EB08006141002487EA115284EA41
:10032000E7731A4340D0009A62B3019A012A4FEA58
:10033000075215DC001B61EB02014FF0004202EA9C
:100340000752CDE90042001C41F5801132462B4690
:1003500000F0CFF903B0BDE8F08F40462146F9E741
:10036000001B61EB0201001C41F5801300185B418A
:100370002018A2F5001747EB030140EAD570B61923
:100380006D4111E06D084FEA360645EAC0754FEA47
:100390000752001B61EB0201001C41F58011490866
:1003A0004FEA30000019514132462B4603B0BDE8F8
:1003B000F04F00F08FB90098012240000023D0EBED
:1003C000020263EBE073009821464FEAE074B8EB59
:1003D000000061EB0401E9E783F000435BE781F093
:1003E000004158E72DE9FE4F81EA030404F0004480
:1003F00021F0004100944FF0000B23F0004350EA3D
:1004000001045ED052EA03045BD0C3F30A54C1F383
:100410000A552C44A4F2F3340194A0FB0254C1F316
:10042000130141F48011C3F3130343F4801301FB60
:10043000024400FB034E840A970A44EA815447EAC7
:100440008357A4FB076802958D0A05FB07854FEAD1
:10045000932C04FB0C542705029D4FEA065847EAEB
:100460001637B5EB08056EEB070C870E920E47EAC0
:10047000811742EA8312A7FB0201B6EB0B0164EB82
:1004800000042B0D43EA0C335E1844EB1C50DA4693
:100490005146E7FB0201C5F313044FEA0B3343EA6D
:1004A00014534FEA0432019C43EA0603A4F10C04FE
:1004B0000294009CCDE900B400F01BF903B0BDE844
:1004C000F08F00200146F9E72DE9F04D81EA0304A1
:1004D00004F0004B21F0004514464FF0000A23F0D1
:1004E000004150EA050220D054EA01021DD0C5F3B4
:1004F0000A570246C5F31303C1F31300C1F30A56AA
:1005000040F4801543F48013A7EB0608101BD64671
:1005100008F2FD3873EB050002D308F1010801E091
:1005200092185B41B8F1000F03DA00200146BDE8E4
:10053000F08D00204FF48011064684460EE0171B14
:1005400073EB050705D3121B63EB050306434CEA67
:10055000010C49084FEA300092185B4150EA01074C
:10056000EDD152EA030012D082EA040083EA0501C9
:10057000084305D0101BAB4106D20122002306E040
:1005800000224FF0004302E06FF0010253101AEB1B
:1005900006004CEB085110EB0A0041EB0B01BDE8E3
:1005A000F04D00F097B800F0004230F000400AD063
:1005B000C10D01F56071C0F3160042EA0151C20895
:1005C00040071143704700200146704701F0004387
:1005D00030B421F0004150EA010206D00A0DA2F524
:1005E0006072C1F31301002A02DC30BC00207047A6
:1005F000440F44EAC104C100E01830BC00EBC25013
:1006000000F031B8202A04DB203A00FA02F1002081
:1006100070479140C2F1200320FA03F31943904040
:100620007047202A04DB203A21FA02F000217047AB
:1006300021FA02F3D040C2F120029140084319464A
:100640007047202A06DBCB17203A41FA02F043EA32
:10065000E07306E041FA02F3D040C2F1200291407B
:100660000843194670470029A8BF7047401C49003D
:1006700008BF20F00100704710B4B0FA80FC00FA07
:100680000CF050EA010404BF10BC704749B1CCF132
:10069000200421FA04F411FA0CF118BF01212143BE
:1006A0000843A3EB0C01CB1D4FEA00614FEA102079
:1006B00042BF002010BC704700EBC350104400291B
:1006C000A4BF10BC7047401C490008BF20F00100C7
:1006D00010BC704710B5141E73F1000408DA401CFA
:1006E00041F1000192185B411A4301D120F0010051
:1006F00010BD2DE9F04D92469B4611B1B1FA81F241
:1007000002E0B0FA80F220329046FFF77BFF044609
:100710000F4640EA0A0041EA0B0153465A46084395
:1007200013D0114653EA010019D0C8F140025046D7
:10073000FFF777FF05460E46504659464246FFF7FB
:1007400061FF084305D0012004E020463946BDE89A
:10075000F08D0020054346EAE0762C4337430A98A3
:100760006305E40AA0EB08000022FD0A44EA4754AE
:100770000A3002D500200146E9E701051019694158
:10078000DDE9084500196941BDE8F04DA2E72DE912
:10079000FE4FC3F30A5701F000450024C1F30A5687
:1007A000C3F31303C1F3130143F4801312EB020AE2
:1007B000A64641F48011009543EB030CA7F1010B11
:1007C00016E0B0EB0A0061EB0C01071E71F10007A7
:1007D00007DA4FF00008D0EB080085F0004568EB21
:1007E0000101171A73EB0107EBD3761E001849417C
:1007F0005E45F6DA50EA010209D0CDE900E50022B3
:1008000013460296FFF775FF03B0BDE8F08F204650
:100810000099F9E7064C074D06E0E06840F0010357
:1008200094E8070098471034AC42F6D3FFF7D8FCA1
:10083000B0680008D06800080EB5C10F80EAE0700B
:100840000844CA07002140F233438DE80E000A46EF
:100850000B46FFF74EFF03B000BD0EB540F233412B
:1008600002910021CDE900110A460B46FFF741FF36
:1008700003B000BD70B5C1F30A5201F00045002479
:10088000C1F3130140F2FF3341F480119A4201DABF
:10089000002070BD40F233439A42A2F2334203DC9F
:1008A0005242FFF7BEFE00E090402C43F1D04042A0
:1008B00070BD000040F2CC60C2F2000000689FED05
:1008C0000B2A90ED090A40F29800B8EE401A9FED0D
:1008D000060AC2F2000021EE000A80EE020A80ED54
:1008E000001A80ED020A7047ACFFB33DA34C65428D
:1008F00010B54EF2180040F2980441F26F21CEF28A
:100900000000C2F20004C3F683210068A16240F235
:10091000CC61C2F200010968206291ED090A9FEDE5
:100920002E2AB8EE401A9FED2B0A84ED001A21EE14
:10093000000A80EE020A94ED012A30EE421A9FED81
:10094000272AB0EEC13AB4EE423AF1EE10FA84ED45
:10095000020A84ED030A84ED041A11DDB5EE401A93
:1009600094ED051AB7EE003ABFEE002AF1EE10FA48
:10097000C8BFB0EE423A33EE011A84ED051A01E029
:1009800094ED051A9FED162A9FED163A21EE021AF4
:1009900094ED0C2A31EE001A31EE422A82EE032A3F
:1009A00040F20801C2F2000191ED003A84ED010A23
:1009B000B8EEC30A84ED0B1A84ED061A84ED0C1A06
:1009C000606222EE000A84ED072A03F079FB84EDD1
:1009D0000D0A10BDACFFB33DA34C65427CD9A040CD
:1009E000DB0FC9406F12833A10B52DED048BB0EECA
:1009F000408AFFF77DFF40F2F000C2F2000080ED78
:100A0000000A38EE400A04F083F940F22404C2F2EE
:100A1000000484ED000A04F0F1F840F2080040F20E
:100A20000401C2F20000C2F200010068096894EDFE
:100A3000008A484300EE100AB8EEC09AFFF73AFF6A
:100A400040F69400C2F2000090ED001A29EE000A70
:100A500030EE410A10EE100AFFF7A5FD41EC100B35
:100A60009FED0F1B05F048F951EC100BFFF7AEFDA1
:100A70009FED0D0A01EE100A71EE000AB5EE401A64
:100A8000F1EE10FAA8BFF0EE410AB0EE480ABDEC54
:100A9000048BBDE8104004F01BBF00BF00BF00BFC7
:100AA00000000060FB211940DB0FC940002181617B
:100AB000016041608160C1600161017570470000A3
:100AC000FEE7000040F2B020C2F2000000F07EBD60
:100AD00040F21030C2F2000000F078BD40F27030F9
:100AE000C2F2000000F072BD40F2D030C2F200004D
:100AF00000F06CBD704700004FF4005001F01CB8CE
:100B0000EFF3108072B600BFFEE7000000000000A7
:100B1000B0B52DED048B9FED2C8A40F2040440F219
:100B20000805C2F20004C2F20005B0EE000AF0EEC1
:100B3000480A2060296004F0CBFE40F6B83000F08F
:100B400031FE9FED220AF0EE480A04F0C1FE28684B
:100B50002168484300EE100AB8EEC09AFFF7AAFEDB
:100B600040F69404C2F2000494ED001A29EE000A43
:100B700030EE410A10EE100AFFF715FD41EC100BA4
:100B80009FED0F1B05F0B8F851EC100BFFF71EFDA1
:100B900000EE100A30EE081AB5EE400AF1EE10FA37
:100BA000A8BFB0EE401A84ED001AFFF7A1FE40F294
:100BB000F000C2F2000080ED000ABDEC048BB0BD75
:100BC00000000060FB211940DB0FC940000000005D
:100BD00040F20C00C2F2000080ED000A04F056B8AA
:100BE00070B582B090F85820012A03D1022108463E
:100BF00002B070BD002201920092026840F2080C1F
:100C0000C5F2000CB2F1A04F0CF1F80508D040F28B
:100C10000043C5F200039A423ED10CF59F6300E009
:100C20002B469B68946823435B0735D44FF4E063FD
:100C3000D1F800E0AA4208BF4FF44073B2F1A04FD0
:100C400008BF4FF440735CF80340BEF1000F24F47A
:100C500060442DD04D6890F838602C4340F2001568
:100C600042F48072C5F2000544EA4634AA424CF8C8
:100C7000034037D1DCF80020DCF800412243D207E2
:100C80003AD15CF80320896840F61F74A24341EA18
:100C90000E01114322E000BFC16D41F02001C1658A
:100CA0000121002280F85820084602B070BD00BF24
:100CB00042F4807140F20012C5F2000291424CF8F9
:100CC00003401BD1DCF80010DCF800211143C907F8
:100CD0001ED15CF8031040F61F7291434CF80310CC
:100CE0000021DEE7DCF80044DCF80055DCF80026E3
:100CF0002C432243D207C4D00021D2E7DCF80024E1
:100D0000DCF80065DCF8001632431143C907E0D077
:100D10000021C6E7F0B581B00022009290F858207B
:100D2000012A03D10221084601B0F0BD0123076862
:100D300080F85830BB685B0736D4D1E900531F26D2
:100D4000C3F3012407EB8404226B03F01F039E40CE
:100D5000B243C5F3846606FA03F31A432263BA6802
:100D6000BB6802F0040203F00803D21840F0BD8013
:100D70000A6807F114030426C2F34064D1F808E0BE
:100D800006EAD25C53F82440C2F304550722AA4075
:100D9000BEF1004F24EA02040CD143F80C401A685B
:100DA00042F000430EE000BFC16D41F02001C1657B
:100DB00001219DE10EFA05F2224343F80C201A6846
:100DC00022F000437B61D1E90435FC68042B5FD13C
:100DD0003A6E3A6E0B68C2F3846293FAA3F6C3F3D9
:100DE000846C6FF3DF43B6FA86F5002B2C464FF682
:100DF000FF7E08BF6446A242C0F2070E0CD13A6ED5
:100E000022F000423A660A6802EA0E03C2F3846CDA
:100E100092FAA2F2B2FA82F57A6E7A6E002BC2F3DF
:100E200084622C4608BF6446A2420CD17A6E22F03E
:100E300000427A660A6802EA0E03C2F3846C92FAF0
:100E4000A2F2B2FA82F5BA6EBA6E002BC2F38462D5
:100E50002C4608BF6446A2420CD1BA6E22F0004272
:100E6000BA660A6802EA0E03C2F3846C92FAA2F22E
:100E7000B2FA82F5FA6EFA6E002BC2F3846208BFF2
:100E80006546AA4231D1FA6E22F00042FA662CE0A1
:100E9000062202EA940205FA02FC0E6807F16005D8
:100EA00055F823404FF20002C0F2FF3206F0F84638
:100EB000224046EA0C06324342F0004245F8232025
:100EC0000A698B6955F8226026F08076334345F82D
:100ED00022300A690B7F55F82260012B26F000763C
:100EE00008BF06F1007645F82260BA68D20750D1F3
:100EF0000D68CA68D7F8B0602B466FF3DF4326EA67
:100F0000030C4FF6FF7602F01804C0F20706E64025
:100F100000242E40C4F27F0446EA0C06A242C7F821
:100F2000B06036D193B195FAA5F2B2FA82F20132ED
:100F300002F01E03092B02F01F0310D801229A4071
:100F400003EB430342EA035315E000BF012202EB27
:100F5000956202F01E030A2B02F01F03EED301225A
:100F600000269A4003EB4303CFF6206606EB0353BB
:100F70001A4342F00073C3F3406607EB86068A68A3
:100F80007569C3F3045307249C40A5439A402A4340
:100F900072610B680021C8F208010B4266D040F272
:100FA000003EC5F2000EAEF500710EF580648F4272
:100FB00004BF40F20034C5F200042146B7F1A04F4F
:100FC00004BF40F20031C5F200018D680022CCF26E
:100FD0002132934205F0E07C04D01022C9F2C00215
:100FE000934245D12A0261D440F20062C5F2000268
:100FF000974202D0B7F1A04F5AD18A6822F0E0722E
:1010000042EA0C0242F400028A6040F21801C2F285
:101010000001096842F663528909C0F23E52A1FB01
:101020000212910901EB41010C2202EB81010091B6
:101030000099002948D000990139009100990029B0
:1010400044D00099013900910099002940D00099BD
:1010500001390091009900293CD000990139009193
:10106000009900294FF00001E5D141E000213FE067
:101070000022CCF25272934208BF15F0807219D050
:101080000021CCF684318B424FF0000108BF15F4EB
:1010900080022DD1B7F1A04F1FD040F20011C5F250
:1010A00000018F4218D1002122E000BF00211FE083
:1010B00000211DE08A6822F0E07242EA0C0242F050
:1010C00080728A60002113E0002111E000210FE00E
:1010D00000210DE000210BE0A646DEF8081021F00B
:1010E000E07141EA0C0141F48001CEF808100021C2
:1010F000002280F85820084601B0F0BDB0B582B09B
:101100000446002001904CB1E06D58B12168886818
:10111000800012D48868C00019D54CE0012002B0CC
:10112000B0BD00BF204600F027F90020206684F8FB
:101130005800216888688000ECD588684FF6C07236
:10114000C5F6FF72104088608868C00033D44FF63F
:10115000C0728868C5F6FF7202F18052104000F13B
:101160008050886040F21800C2F20000006842F629
:1011700063528009C0F23E52A0FB02029009022293
:1011800002EB400001900198A8B100BF019801381E
:101190000190019878B1019801380190019850B1FF
:1011A000019801380190019828B101980138019007
:1011B00001980028EAD18868C00009D4E06D40F0A9
:1011C0001000E065206E40F001002066012000E084
:1011D00000208A68E36D02F0040203F01003D218C5
:1011E000E26D40F0818022F481720232E2658A6809
:1011F000D20729D140F2001341F48072C5F20003F6
:1012000040F2080C9A42C5F2000C73D1DCF80030B1
:10121000DCF800211A43D20716D10CF1F8024FF482
:10122000E063D4F804E0914208BF4FF44073B1F199
:10123000A04F08BF4FF440735CF8032022F47C12E7
:1012400042EA0E024CF80320627FE36B43EA42322B
:10125000D4E902C31A4394F8243042EA0C02012B69
:1012600042EA034207D1D4F828C00023CFF6FE7328
:1012700003EB4C431A43E36A33B103F47873D4F8B5
:1012800030C01A4342EA0C02D1F80CC044F2070302
:10129000CFF6F07303EA0C031A43CA600A69636B62
:1012A00022F040621A430A618A68120753D494F804
:1012B0003820237F520042EA833CCB6844F202028A
:1012C00023EA020242EA0C02CA6022690B69FAB1FF
:1012D00043F480330B61D1F8C0C043F6FF732CEAAE
:1012E00003031A431CE000BF42F010010120E16536
:1012F00002B0B0BDDCF800E4DCF80025DCF8003614
:1013000042EA0E021A43D2073FF487AF9CE700BFC0
:1013100023F480320A61D1F8C02043F6FF739A4368
:10132000C1F8C02094F840300A69012B10D140F276
:10133000FD7322EA030CD4E91132D4E913E543EA40
:101340000C031A4342EA0E022A4342F0010201E072
:1013500022F001020A6162690B6B012A23F00F027D
:1013600002D1236A013B1A430A63E16D012262F351
:101370000101E16502B0B0BDF0B59BB004460020AC
:101380001A90CDE91800CDE9160001A85421FEF706
:1013900077FF206840F20041C5F2000188426FD01B
:1013A00040F20011C5F20001884200F0A380B0F1C4
:1013B000A04F40F009814FF4004001904FF00050E1
:1013C000129001A800F024FF002818BFFFF798FB37
:1013D00040F2D001C2F200014A6841F24C00C4F26E
:1013E0000200531C4B6042B9016841F40051016096
:1013F000016801F4005100910099016816AD41F0B7
:10140000040101600168032701F0040100910099C3
:101410000168002641F0010101600068294600F0E2
:101420000100009000980820169040F20040C4F699
:10143000000000F580601797189600F089FB4FF0C8
:1014400090402946CDE91677189600F081FB40F2CE
:10145000B0250820C2F20005C4F202000521802256
:101460004FF4007385E8430005F114004FF4006762
:101470004FF0200CC5E9036280E888109BE000BFB4
:101480004FF4803001904FF00040139001A800F01D
:10149000BFFE002818BFFFF733FB41F24C00C4F237
:1014A00002000168002641F480410160016801F4F6
:1014B000804100910099016841F0020101600068DB
:1014C00016A900F002000090009802201690032058
:1014D000179040F20040C4F60000189600F038FB68
:1014E0000820C4F2020040F270352830C2F2000534
:1014F000252153E04FF4004001904FF0005012902E
:1015000001A800F085FE002818BFFFF7F9FA40F2A5
:10151000D001C2F200014A6841F24C00C4F202005C
:10152000531C4B6042B9016841F4005101600168ED
:1015300001F4005100910099016816AD41F00101DC
:1015400001600168032701F0010100910099016821
:10155000002641F0020101600068294600F0020007
:1015600000900098C02016904FF090401797189662
:1015700000F0EEFA0420CDE9160740F20040C4F670
:1015800000002946189600F0E3FA0820C4F2020091
:1015900040F210351430C2F20005242180224FF4AD
:1015A00000734FF4006728606960AE60EE602A61E6
:1015B0006B61AF61EE6128462E6200F05DF808B104
:1015C000FFF79EFA6565AC621BB0F0BDB0B5D0E91F
:1015D00010C30268DCF8001003F01F030424D2F8E3
:1015E00000E09C400C4218BF1EF0040522D10224EA
:1015F0009C400C4218BF1EF0020529D1D9400907B2
:1016000024D51EF0080108BFB0BD116821F00E01FD
:101610001160012101FA03F2CCF80420C16380F8C3
:101620002510416B002280F8242079B1BDE8B0403C
:10163000084700BF1168890603D4116821F004012E
:101640001160CCF80440016B0029EFD1B0BD00BFA0
:101650001168890606D4116821F00A011160012180
:1016600080F82510CCF80440C16A0022002980F8D7
:101670002420DBD1EAE7000000284FF0010100F050
:101680008E802DE9F04740F2000CC4F2020C036892
:101690004FF6F8320CF5816ECBF6FD72734538BF0C
:1016A00002F580624CF6CD441A44CCF6CC44A2FB41
:1016B00004286FF0070252FA83F2A2FB04290CF50A
:1016C00080656FF00304D0E90262D0F810A03CBF3F
:1016D0000025C4F2020504EA9804C0E9105402256A
:1016E00080F825501D6847F6F07725EA070737434D
:1016F0003A43476942EA0A0285693A43C7692A437D
:10170000056A3A432A431A600CF50262734538BFF2
:101710000CF50062A3180CF50862C264C9F3041248
:1017200040F6840C01FA02F2B6F5804FC4F2020CC6
:101730008364026506D1002141601960CCF8002065
:101740001EE000BF41685FFA81FE013903294FF0B6
:101750000001C3F800E0CCF8002011D8AEF101027E
:101760000CEB820747F87C1F02F01F01012202FAEE
:1017700001F30CF1BC023946CCF8C03002E000BFE6
:101780000022002300F1540C8CE80E0000210122FD
:10179000C16380F8252080F82410BDE8F047084692
:1017A00070470000B0B5044600F0C6FA054640F2A6
:1017B0001000C2F200004068611C18BF044400BF62
:1017C00000F0BAFA401BA042FAD3B0BD70B5D8B150
:1017D000044690F85C0028B9002084F85D0020469B
:1017E00000F01EF92068816921F01001816100F08C
:1017F000A3FA054620688169090707D500F09CFA1D
:10180000401B0B28F6D312E0012070BD816941F026
:101810000101816100F090FA054600BF20688169EE
:10182000C9070DD100F088FA401B0B28F6D3206EB3
:10183000032140F001002066012084F85C1070BD97
:10184000826946F2004CC4F2000C42F0020260458C
:10185000826102D16268CCF80021227C8369012A6E
:1018600023F0400318BF40338361627C8369012AFF
:1018700023F4804308BF03F580438361A27C83691E
:10188000012A23F4805318BF03F5805383618269D2
:10189000D4E902E322F4407545EA0E0585618569C5
:1018A00025F0A4058561056925F0100505619BB14A
:1018B000012B0DD0022B09D08569032B45F0800543
:1018C0008561056945F01005056105D1202300E01B
:1018D000042385692B43836104F114052ACD226A10
:1018E0005E1E6FF0FF0303EB052545EA4665013AEE
:1018F0002A430025CFF6FF7505EB01411143BEF5E4
:10190000407FC16110D1D4E909E2D4E90B61013A09
:1019100003EB06231A436FF00F0303EB011111438E
:1019200005EB0E421143C160D4E90D13E26BD0F810
:10193000C0603243C0F8C0200CF580660CF58042D0
:10194000B04204BF4AF25072C4F200020CF50066C5
:10195000B04208BF02F5D4622264D0F8806026F459
:10196000F81646EA0141C0F8801002F17001616486
:10197000D0F8801021F0706141EA0361C0F8801056
:1019800002F1B000A06402F5C470E06402F51870C2
:10199000206502F51E70606502F55470002100BFDD
:1019A000C2E90011C2E90211C2E90411C2E906113B
:1019B000C2E90811C2E90A11C2E90C11C2E90E110B
:1019C000C2E91011C2E91211C2E91411C2E91611DB
:1019D000C2E91811C2E91A11C2E91C11C2E91E11AB
:1019E000C2E92011C2E92211C2E92411C2E926117B
:1019F000C2E92811C2E92A11C2E92C11C2E92E114B
:101A0000C2E93011C2E93211C2F8D010D432824298
:101A1000C6D300200121A065206684F85C1070BD4B
:101A200010B59CB0044600201B90CDE91900CDE90B
:101A3000170002A85421FEF723FC206846F6000197
:101A4000C4F20001884237D046F20041C4F20001DE
:101A500088426DD14FF4805002904FF0007010908A
:101A600002A800F0D5FB002818BFFFF749F840F2A4
:101A7000F401C2F200010A6841F24C00C4F2020013
:101A8000531C0B6042B9C16841F00071C160C1686C
:101A900001F0007101910199016841F001010160BB
:101AA000006800F00100019001984FF4C0501790B9
:101AB0004FF0904032E000BF4FF4805002904FF062
:101AC0000070109002A800F0A3FB002818BFFFF7D9
:101AD00017F840F2F401C2F200010A6841F24C002A
:101AE000C4F20200531C0B6042B9C16841F000719E
:101AF000C160C16801F0007101910199016841F074
:101B000002010160006800F00200019001984FF4AA
:101B10008250179040F20040C4F600000221189154
:101B20000021CDE9191109211B9117A900F010F826
:101B30001CB010BD7047000040F21441C4F2010116
:101B40000A68024214BF08607047FFF7F3BF000045
:101B50002DE9F04F84B08E4641F20042C4F60002F7
:101B6000DEF8004006219042019008BF0521002CBC
:101B7000009100F0D7800198002500F138424FEA2B
:101B8000B2230098012700264FF00008052B38BF2C
:101B900018460090CDF808E00EE000BFDEF80040E7
:101BA00008F1010834FA07F106F1020607F101070E
:101BB00005F1040500F0B680A7F1010A012000FA42
:101BC0000AF314EA0309E9D0DEF804C00CF0030BB1
:101BD000ABF10104012C17D80198744681680322E7
:101BE000E468B2409143B4402143816041684FEAC8
:101BF000480E9943CCF3001303FA0AF30446D0438A
:101C0000194361600CE000BF0321B140019CC8434F
:101C1000BBF1030FB64603D1B6464FF0030B23E0EA
:101C2000E168029A01409368BBF1020F03FA0EF3D8
:101C300041EA0301E16017D16FF0030101EA5A01A3
:101C4000214405F01C040F23D1F820C003FA04FB43
:101C500013692CEA0B0CA34043EA0C03019C0B62B2
:101C6000D2F804C00CF0030B21680BFA0EF201400D
:101C700011432160DDF808E01CF4403F8ED041F2B2
:101C80006000C4F20200016840F2004C41F0010122
:101C900001600168C4F2010C01F001010391039994
:101CA0002AF003014FF6084A6144CFF6FF7A05F0A7
:101CB0000C030F2051F80A2000FA03F40098A24305
:101CC00000FA03F31A4341F80A20DCF80810DEF8A2
:101CD000042041EA090340F20C40D40258BF21EA33
:101CE0000903CCF80830C4F201000168940241EA0B
:101CF000090358BF21EA09030360DCF804109403C8
:101D000041EA090358BF21EA0903CCF80430DCF8A2
:101D10000010D20341EA090358BF21EA0903CCF8B5
:101D200000303BE704B0BDE8F08F00001823002A24
:101D300008BF2823C150704740F68C00C2F2000053
:101D40000068704790F84120202A03D190F8402085
:101D5000012A01D102207047242280F84120026824
:101D6000136823F001031360136823F48053136096
:101D7000136819431160116841F0010111602021BD
:101D800080F84110002180F840100846704700009C
:101D900090F84120202A03D190F84020012A01D157
:101DA00002207047242280F841200268136823F043
:101DB00001031360136823F4706343EA0121116087
:101DC000116841F001011160202180F841100021CB
:101DD00080F8401008467047002804BF0120704773
:101DE00010B5044690F8410028B9002084F840005E
:101DF000204600F049F8242084F8410094E80910B6
:101E0000E2680168012A21F00101016023F070619C
:101E10000161816821F40041816003D14CF40041EB
:101E2000816009E04CF40441022A816004D14168D8
:101E300041F4006103E000BF416821F400614160AA
:101E4000416804F1100C41F0007141F4004141601F
:101E5000C16821F40041C1609CE80E10114341EAC1
:101E60000321C160216A41EA0C010160016841F06F
:101E70000101016000202021606484F8411020638A
:101E800084F8420010BD000010B59CB0044600204C
:101E90001B90CDE91900CDE9170002A85421FEF7E7
:101EA000EFF9206845F60001C4F20001884237D0FE
:101EB00045F20041C4F2000188425FD14020029007
:101EC00002A800F0A5F9002818BFFEF719FE41F29C
:101ED0004C04C4F20204206817A940F002002060FC
:101EE000206800F00200019001984FF4C070179034
:101EF000122018900020CDE9190004201B9040F218
:101F00000040C4F60000FFF723FEE06840F4001034
:101F1000E060E06800F40010019001981CB010BD72
:101F20008020029002A800F073F9002818BFFEF785
:101F3000E7FD41F24C04C4F20204206817A940F006
:101F400001002060206800F00100019001984FF42A
:101F500040701790122018900020CDE9190004203D
:101F60001B904FF09040FFF7F3FDE06840F48000D5
:101F7000E060E06800F48000019001981CB010BDA2
:101F800040F2100040F68C01C2F20000C2F20001E3
:101F900040680A68104408607047000080B503205C
:101FA00000F088F8002000F009F800281CBF01208C
:101FB00080BD00F029F8002080BD000070B540F21F
:101FC0001006C2F200067168E1B1044640F2180042
:101FD000C2F200004FF47A720068B2FBF1F1B0FB7C
:101FE000F1F000F0CBFE0F2C4FF0010508D838B906
:101FF0004FF0FF3021460022002500F02FF834601A
:10200000284670BD012070BD82B041F25800C4F274
:102010000200816841F001018160816801F00101E5
:1020200001910199016841F080510160006800F060
:1020300080500090009802B000F0E0B8002848BF3F
:10204000704700F01F01012202FA01F14EF2001266
:102050004009CEF2000242F82010704710B54EF64B
:102060000C5CCEF2000CDCF80030C3F3022E8EF0D4
:102070000704042C28BF0424BEF103034FF0FF3EE5
:102080000EFA04F438BF0023A14399400EFA03F37B
:102090009A43114300F00F02043A624409010C32E2
:1020A00000F16043B0F1FF3FC8BF03F56442117017
:1020B00010BD00004EF60C51CEF200010A684FF63A
:1020C000FF031A4060F30A2242F0806040F0FD7086
:1020D00008607047B0F5007F42D0002840F0808053
:1020E00047F21400C4F2000050F8141CC26E01F450
:1020F000C06122F48072B1F5806FC2662ED150F8B3
:10210000141C012262F34A2140F8141C40F2180109
:10211000C2F200010968322251434DF68362C4F2D3
:102120001B32A1FB0212910C0268520511D54A1C08
:102130000FD0026852050CD559B10268520508D576
:10214000012906D00268520503D50229A1F1040134
:10215000EAD10068400544BF032070470020704763
:1021600047F21400C4F2000050F8141CC26E01F4CF
:10217000C06142F48072B1F5806FC266EED150F852
:10218000141C012262F34A2140F8141C40F2180189
:10219000C2F200010968322251434DF68362C4F253
:1021A0001B32A1FB0212910C0268520511D54A1C88
:1021B0000FD0026852050CD559B10268520508D5F6
:1021C000012906D00268520503D50229A1F10401B4
:1021D000EAD10068400544BF03207047BEE700BF56
:1021E00047F21400C4F2000050F8141C022262F3FB
:1021F0004A2140F8141C00207047000047F20800F4
:10220000C4F20000016841F48041016070470000A1
:102210002DE9F04182B00446807841F2880600073B
:10222000C4F2020602D400202FE000BF56F8300CA2
:1022300010F080580BD156F8300C40F0805046F822
:10224000300C56F8300C00F080500190019847F2A5
:102250000007C4F20007386840F480703860FFF768
:102260006BFD05463868C00500F10C81FFF764FD81
:10227000401B0228F6D90320B8F1000F05D156F80B
:10228000301C21F0805146F8301C2168CA0717D154
:102290008A071DD44A0723D40A0729D4CA062FD493
:1022A0008A0635D44A063BD40A0641D4CA0547D427
:1022B0008A034DD48A0553D44A0559D467E000BF38
:1022C0003268636822F003021A4332608A07E1D55C
:1022D0003268A36822F00C021A4332604A07DBD549
:1022E0003268E36822F030021A4332600A07D5D51B
:1022F0003268236922F0C0021A433260CA06CFD581
:102300003268636922F440721A4332608A06C9D582
:102310003268A36922F440621A4332604A06C3D588
:102320003268E36922F440521A4332600A06BDD58E
:102330003268236A22F440421A433260CA05B7D594
:102340003268636A22F440321A4332608A03B1D59C
:102350007269A36A22F003021A4372618A05ABD53F
:102360003268E36A22F440221A4332604A050ED5ED
:102370003268236B22F440121A43B3F5801F326097
:1023800005D156F87C2C42F4801246F87C2C0A05C4
:102390000ED53268636B22F440021A43B3F5800F06
:1023A000326005D156F87C2C42F4801246F87C2C21
:1023B000CA040ED53268A36B22F040721A43B3F1FF
:1023C000807F326005D156F87C2C42F4801246F8AA
:1023D0007C2C8A040ED53268E36B22F040621A43EB
:1023E000B3F1006F326005D156F87C2C42F48012B4
:1023F00046F87C2C4A040ED53268236C22F04062E9
:102400001A43B3F1006F326005D156F87C2C42F4C8
:10241000801246F87C2C0A040ED53268636C22F0D8
:1024200040521A43B3F1805F326005D156F87C2CDC
:1024300042F4803246F87C2CCA030ED53268A36C75
:1024400022F040421A43B3F1804F326005D156F872
:102450007C2C42F4803246F87C2C49030ED57169FD
:10246000E26C21F440111143B2F5001F716105D1F6
:1024700056F87C1C41F4801146F87C1C02B0BDE883
:10248000F08100BFB06810F4407010D0216D884218
:102490000BD0B068B16820F4407041F48031B16075
:1024A000B16821F48031B160B060C0070CD1B06870
:1024B000216D20F440700843B0600020B8F1000F97
:1024C0007FF4E3AEDBE600BFFFF736FC054641F2E2
:1024D000883700BFB0688007E9D4FFF72DFC401BA8
:1024E000B842F7D9C7E600002DE9F04700286DD0C3
:1024F00042F2000AC4F2020A0446DAF800000D466D
:1025000000F00F0088420CD2DAF8000020F00F0033
:102510002843CAF80000DAF8000000F00F00A842D3
:1025200054D1216841F20808C807C4F2020803D157
:10253000880740F1D880BDE0606802283AD00328BF
:1025400040D158F8082C920140D5D8F80420D8F88A
:10255000043042F2004702F00302C3F30313C0F257
:10256000F4070133032A04BF43F20067C0F26E1779
:10257000D8F80420B7FBF3F3D8F80470C2F30622AE
:102580005A43C7F34163022707EB4303B2FBF3F25D
:102590004BF20043C0F2C4439A4261D9D8F80020FC
:1025A00012F0F00F51D089075AD5A168002957D1F0
:1025B0004BE000BF58F8081C89035CBF0120BDE850
:1025C000F08707E058F8081C490503D40120BDE84E
:1025D000F08700BFD8F8001001F00C0104293FD0AB
:1025E000D8F8001001F00C01082939D0D8F80010F3
:1025F00001F00C010C2933D1D8F80410D8F80420CC
:1026000042F2004301F00301C2F30312C0F2F403EB
:102610000132032904BF43F20063C0F26E13D8F8FD
:102620000410B3FBF2F2D8F80430C1F30621514391
:10263000C3F34162022303EB4202B1FBF2F14BF21E
:102640000042C0F2C44291420AD9D8F800100822D0
:1026500062F307114FF00109C8F8001002E000BF53
:102660004FF00009D8F8001021F003010843C8F822
:102670000000FFF761FB064641F28837D8F80000FA
:10268000616800F00C00B0EB810F07D0FFF754FB3E
:10269000801BB842F2D90320BDE8F0872168880783
:1026A00008D4B9F1000F1ED0D8F8000020F0F000D7
:1026B00017E000BF480705D5D8F8000040F4E060F7
:1026C000C8F80000080706D5D8F80000072262F312
:1026D0000D20C8F80000D8F80000A26820F0F00033
:1026E0001043C8F80000DAF8000000F00F00A8421C
:1026F0001BD9DAF8000020F00F002843CAF80000C8
:10270000FFF71AFB064641F2883700BFDAF80000EF
:1027100000F00F00A84207D0FFF70EFB801BB84265
:10272000F4D90320BDE8F0872168480707D5D8F819
:102730000000E26820F4E0601043C8F800000807D9
:1027400008D5D8F80000216920F4605040EAC100A3
:10275000C8F80000D8F8000042F20041C0F2F401CD
:1027600000F00C00042808462DD0D8F8000000F036
:102770000C00082843F20060C0F26E1023D0D8F895
:10278000002002F00C020C2A1CD1D8F80420D8F842
:10279000043002F00302C3F303130133032A08BF1A
:1027A0000146D8F80400B1FBF3F1D8F80420C0F3D7
:1027B00006204843C2F34161022202EB4101B0FB13
:1027C000F1F000E00020D8F8001046F66002C1F3F6
:1027D0000311C0F60002515C40F2180201F01F0123
:1027E00020FA01F140F21000C2F200000068C2F2CB
:1027F00000021160BDE8F047FFF7E0BB40F21800AF
:1028000041F20801C2F20000C4F202010068096846
:1028100046F67002C1F30221C0F60002515C01F0DD
:102820001F01C8407047000040F2180041F2080143
:10283000C2F20000C4F202010068096846F67002A4
:10284000C1F3C221C0F60002515C01F01F01C84073
:102850007047000041F20C01C4F2020151F8040C6F
:1028600042F20042C0F2F40200F00C0004281046CC
:1028700008BF704751F8040C00F00C00082843F220
:102880000060C0F26E1021D051F8043C03F00C033C
:102890000C2B1CBF00207047D1F800C00B680CF057
:1028A000030CC3F303130133BCF1030F08BF02464B
:1028B0000868B2FBF3F20968C0F306205043C1F385
:1028C0004161022202EB4101B0FBF1F070470000D0
:1028D0002DE9F04182B0002800F00681044600781E
:1028E00041F20006C007C4F2020655D120788007E5
:1028F00074D42078000700F197802078400700F119
:10290000B7802078800600F10781E569002D00F08E
:102910003082B06800F00C000C2840F05981012D85
:1029200000F0E280F068216A00F003028A4240F081
:10293000DB80626A6FF00F0300F0F00103EB02121C
:10294000914240F0D180A16A00F4FE42B2EB012F27
:1029500040F0CA80E16A00F07842B2EBC16F40F00B
:10296000C380226B0023CFF6E07303EB025200F426
:10297000C0016FF31402914240F0B680616B4FF0DA
:102980007E4202EB016100F0C06001F07E418842AE
:1029900040F0AA80EDE100BFB06800F00C01F068E3
:1029A00008295BD0032281F00C0122EA00000844D0
:1029B000B0FA80F0400951D16068B0F5803F07D08F
:1029C000B0F5A02F40F0DA80306840F4802030600D
:1029D000306840F480303060DBE000BFB068F16800
:1029E00000F00C00042869D001F0030180F00C0015
:1029F00081F002010844B0FA80F040095ED1E1683C
:102A00003068002900F0D28040F480703060FFF719
:102A100093F905463068400500F1FC80FFF78CF91A
:102A2000401B0228F6D92EE16169D6F894000029EE
:102A300000F0908040F00100C6F89400FFF77CF9A8
:102A4000054600BFD6F8940080073FF556AFFFF764
:102A500073F9401B0228F5D915E100BF30688003E7
:102A60007FF544AF606800287FF440AF3CE000BFD2
:102A7000B06D10F0805808D1B06D40F08050B06556
:102A8000B06D00F080500190019847F20007C4F249
:102A900000073868C0052BD4386840F4807038606F
:102AA000FFF74AF9054600BF3868C00520D4FFF794
:102AB00043F9401B0228F7D9E5E000BF3068400524
:102AC00001D5E06880B17068216920F0FE4040EADD
:102AD0000160706040F21000C2F200000068FFF771
:102AE0006DFA00283FF405AF012002B0BDE8F08187
:102AF000A068012808D0052840F0AA80D6F89000E8
:102B000040F00400C6F89000D6F8900040F00100B4
:102B1000C6F89000A9E000BFA169D6F89800002986
:102B200000F0808040F00100C6F89800FFF704F93B
:102B3000054600BFD6F8980080073FF5E6AEFFF7E0
:102B4000FBF8401B02284FF00300F3D902B0BDE8A8
:102B5000F08100BF20F00100C6F89400FFF7ECF808
:102B6000054600BFD6F8940080077FF5C6AEFFF794
:102B7000E3F8401B0228F5D985E000BF3168002842
:102B800021F480313160316821F48021316000F01E
:102B90007F80FFF7D1F80546306880033FF5A6AE89
:102BA000FFF7CAF8401B6428F6D96CE020F4807067
:102BB0003060FFF7C1F80546306840057FF599AEF3
:102BC000FFF7BAF8401B02284FF00300F4D9BDE725
:102BD000306820F080703060FFF7AEF8022D0546B7
:102BE0000CD100BF3068800140F17E80FFF7A4F86F
:102BF000401B02284FF00300F4D9A7E7306880019A
:102C000040F1B080FFF798F8401B02284FF0030016
:102C1000F4D99BE77068216920F0FE4040EA01602A
:102C2000706066E620F00100C6F89800FFF784F8AF
:102C3000054600BFD6F8980080077FF566AEFFF71F
:102C40007BF8401B02284FF00300F3D97EE700BF5A
:102C5000D6F8901021F00101C6F89010D6F8901027
:102C600021F00401C6F8901010B3FFF765F805468F
:102C700041F28837D6F8900080072BD4FFF75CF834
:102C8000401BB842F6D9032002B0BDE8F08100BF76
:102C9000FFF752F8054600BF306880037FF526AE87
:102CA000FFF74AF8401B64284FF00300F4D94DE7C2
:102CB000FFF742F8054641F2883700BFD6F890008A
:102CC000800707D5FFF738F8401BB8424FF00300E4
:102CD000F4D93BE7B8F1000F7FF413AEB06D20F0EC
:102CE0008050B0650DE600BFF06848F20C01C0F2FC
:102CF0009F1104F1200700EA010C8ECF6FF00F0046
:102D0000D4E90C5400EB02100022CFF6E07241EA45
:102D10000C0102EB055208436FF314024FF07E459D
:102D200040EA032005EB0465104305F07E4540EAC8
:102D3000C7602843F060306840F080703060F06811
:102D400040F08070F060FEF7F7FF044630688001C5
:102D50000FD4FEF7F1FF001B02284FF00300F5D956
:102D6000F4E600BFF0684FF6FC71CFF6EE61084064
:102D7000F060002002B0BDE8F0810000411E00209C
:102D8000B0EB116F1CBF012070474EF21002CEF263
:102D9000000251604EF62351CEF20001F0230B7079
:102DA0000721906011607047B0B590F83C20012A6F
:102DB00004BF0220B0BDD1E90232D1E900CE22F435
:102DC0007C5223F4705343EA020448F2FF73CEF6B8
:102DD000F0730EEA0302224303F5006404EA0C04D4
:102DE00042EA040C0C6903F5C05222404C6942EAE5
:102DF0000C02224303F5605422400C6B03F5F043B0
:102E000023401A438B6940F2000CCC69CEF6FF7C5C
:102E10000CEA034C1443026842F60043C4F2010377
:102E20009A4244EA0C030BD045F20004C4F20104B8
:102E3000A24205D043F20044C4F20104A24217D1D9
:102E40004FF6FF74CDF60F4403EA040ED1E9084CA7
:102E5000D1E90A310025CDF6F04505EA035343EAEE
:102E60000E0324F008552B432CF000552B430B4345
:102E70000021536480F83C100846B0BDB0B504464C
:102E800090F83C00012804BF0220B0BD0D46206828
:102E9000D1E90021AB684FF0010C84F83CC002F08E
:102EA00045F82068816DD5E9042321F0E7012D7BE9
:102EB00019431143012D08BF41F0200141F00101E8
:102EC0008165002084F83C00B0BD00000168886D79
:102ED00040F0010200208A657047000070B590F84C
:102EE0003C20012A4FF0020265D080F83D200268A4
:102EF00042F600435468D2F808C0C4F2010345F218
:102F0000000E9A42C4F2010E18BF72452CD14D68D2
:102F100024F470042C434FF68F75CFF6FF550E68DE
:102F20002C4042F6FF35C4F201053443AA425460F6
:102F30000EDC40F2FF73C4F200039A421CDCB2F1D3
:102F4000804F2DD040F20043C4F2000326E000BFC2
:102F500043F6FF74C4F20104A24219DC9A421FD066
:102F600043F2004318E000BF43F20045C4F20105FC
:102F7000AA42CCD0CFE700BF40F60003C4F2000362
:102F80009A420DD040F60043C4F2000306E000BFB1
:102F9000724505D044F20003C4F201039A4204D101
:102FA00089682CF08003194391600121002280F888
:102FB0003D1080F83C20104670BD000041B108294A
:102FC00010D0042914BF00F1470200F145020BE0C4
:102FD00090F84420012A1CBF01207047022280F88B
:102FE000442013E000F146021278012A1CBF0120A0
:102FF00070470222082907D0042914BF80F847200F
:1030000080F8452002E000BF80F84620026801F009
:103010000F000421136A01FA00F023EA0001116293
:10302000116A08431062506C42F6FF31C4F201018C
:1030300040F400408A4250640EDC40F2FF70C4F25B
:103040000000824218DCB2F1804F2DD040F20040E7
:10305000C4F2000026E000BF43F6FF70C4F2010096
:10306000824215DC42F60040C4F2010082421BD0CD
:1030700043F2004014E000BF40F60000C4F200003C
:10308000824211D040F60040C4F200000AE000BFC6
:1030900045F20000C4F20100824205D044F2000073
:1030A000C4F2010082420CD190680721C0F20101F4
:1030B000014006294FF0000008D0B1F5803F08BF5D
:1030C0007047106840F00100106000207047000059
:1030D000002804BF0120704710B5044690F83D0059
:1030E00028B9002084F83C00204600F023F8022094
:1030F00084F83D002068211D01F072FE012084F853
:10310000480084F83E0084F83F0084F8400084F8CA
:10311000410084F8420084F8430084F8440084F8B5
:10312000450084F8460084F8470084F83D000020FC
:1031300010BD000082B0006843F20041C4F20101FA
:10314000884215D042F60041C4F2010188421CD1E8
:1031500041F26000C4F20200016841F400610160C4
:10316000006800F400600190019802B0704700BF51
:1031700041F26000C4F20200016841F400510160B4
:10318000006800F400500090009802B07047000002
:1031900080B590F83C20012A4FF0020200F09880A0
:1031A00080F83D20D0F800C08822DCF80830CFF647
:1031B000CE721A40CCF808200B68B3F5005F0DDA28
:1031C0003F2B21DD5F2B33DD602B00F08380702BE4
:1031D00000F0A280B3F5805F73D0E7E02F22C0F249
:1031E0001002934218DD4F21C0F210018B4247DDDF
:1031F0005021C0F210018B4257D06021C0F2100163
:103200008B4252D070214BE01F2B41DC002B4CD065
:10321000102B4AD0CAE000BFB3F1101F3EDAB3F55D
:10322000005F00F08D80B3F5801F3ED0BEE000BF90
:10323000402B00F09980502B40F0B880D1F804E08A
:10324000C968DCF82030DCF8202022F00102CCF83C
:103250002020DCF8182022F0F00242EA011123F0CD
:103260000A0242EA0E02CCF81810CCF82020DCF852
:1032700008104FF68872CFF6CF72114057311EE01A
:103280003021C0F210018B420FD0402108E000BF76
:10329000202B0AD0302B08D088E000BF05D0202199
:1032A000C0F210018B4240F08180DCF808104FF62C
:1032B0008872CFF6CF721140194341F00701CCF864
:1032C00008100022012180F83D10002180F83C10F8
:1032D000104680BDD1F804E0C968DCF82030DCF885
:1032E000202022F01002CCF82020DCF8182022F454
:1032F000704242EA013123F0A00242EA0E12CCF8F9
:103300001810CCF82020DCF808104FF68872CFF6A1
:10331000CF7211406731D2E7D1E901E3C968DCF827
:10332000082043EA0E0322F47F4243EA01211143BD
:10333000CCF80810DCF8081041F07701BFE700BFB7
:10334000D1E901E3C968DCF8082043EA0E0322F45E
:103350007F4243EA01211143CCF80810DCF8081041
:1033600041F48041ABE700BFD1F804E0C968DCF864
:103370002030DCF8202022F00102CCF82020DCF8FC
:10338000182022F0F00242EA011123F00A0242EA78
:103390000E02CCF81810CCF82020DCF808104FF6FC
:1033A0008872CFF6CF721140473188E7012289E752
:1033B000002804BF012070472DE9F047044690F82B
:1033C0003D000D4628B9002084F83C00204600F05E
:1033D0004BF8022084F83D0020684BF6F8728168B3
:1033E000CFF6FE7211408160211D01F0F9FC2068CA
:1033F0004FF6FF7881688269D0F820C0D5E9003E99
:10340000D5E9026A43EA0109AB6922EA080246EA01
:1034100003234FF6FC46B343D5E9076742EA0A02A5
:1034200029691A4342EA062242EA01112CF0AA0253
:103430006B6942EA0E0241EA073142EA0312C0F820
:10344000089081610262012084F8480084F83E00FF
:1034500084F83F0084F8440084F8450084F83D0077
:103460000020BDE8F08700002DE9F04186B000683B
:1034700040F20041C4F2000100268842CDE9046612
:10348000CDE90266019649D0B0F1804F40F09580B9
:1034900041F24C00C4F20200C1680DF1040841F091
:1034A0000101C160C168022601F00101009100998B
:1034B0000168002741F00101016001684FF090446C
:1034C00001F0010100910099016841F002010160E1
:1034D0000068414600F00200009000982020019012
:1034E0004FF090400296CDE903770596FEF730FB4A
:1034F0004FF4816001A9C1C140F200400125C4F62A
:103500000000414604970595FEF722FB4FF400406A
:1035100001A9C1C1CDE904754BE000BF41F24C00E7
:10352000C4F20200C16801AC41F00201C160C1688F
:10353000022701F0020100910099016841F00101A8
:103540000160016801F0010100910099016841F0FA
:1035500002010160016801F0020100910099016817
:1035600041F0080101600068214600F00800009069
:103570000098102001904FF09040CDE90276CDE9FF
:103580000467FEF7E5FA40F200451120C4F6000595
:10359000CDE9010728462146CDE903660597FEF7E8
:1035A000D7FA042005F50064CDE90107CDE90366EB
:1035B000059701A92046FEF7CBFA06B0BDE8F081D9
:1035C00080B590F83E2090F83F3090F844E090F8B5
:1035D00045C004290AD0B9B9012A4FF0010208BF39
:1035E000BEF1010F34D0104680BD00BF012B4FF05B
:1035F000010208BFBCF1010FF5D1022180F83F1094
:1036000080F8451000681EE0012A4FF0010208BF53
:10361000012BE8D1BEF1010FE5D1BCF1010FE2D1E0
:10362000022280F83E2080F83F2080F8442080F875
:10363000452091B10068016A21F001010162016A2F
:1036400041F00101016210216FF0100209E000BF9A
:10365000022180F83E1080F84410006801216FF0CC
:103660000102036A1A400262026A114301620168A0
:10367000002241F001010160104680BDF0B587B025
:10368000006843F20042C4F2010200219042CDE9F9
:103690000511CDE9031102913ED042F60041C4F27A
:1036A0000101884258D141F24C00C4F20200016885
:1036B00040F2004441F0040101600168C4F60004D6
:1036C00001F0040101910199016802AD41F002018C
:1036D00001600068022600F00200019001980720B6
:1036E0000290002704F5806029460396CDE904770F
:1036F0000696FEF72DFA4FF4C04002A9C1C106207C
:103700000690204629460597FEF722FA4FF400401E
:1037100002A9C1C1059719E041F24C00C4F20200B0
:10372000026842F004020260006800F004000190A8
:1037300001984FF4EE5002900220CDE9030140F2CF
:103740000040C4F6000000F5806405910420069056
:1037500002A92046FEF7FCF907B0F0BD2DE9F041C3
:1037600090F83C30012B04BF0220BDE8F0814FEA05
:10377000B202052A00F2A281DFE812F0060054002E
:10378000AE0008016201A80103681D6A1A6AA3F16C
:10379000804622F001021A621A46D3F8048052F8D9
:1037A00018EF8F68A6F59636D1F800C025F002050F
:1037B0004FEAB626092E45EA07050BD80127B74080
:1037C00040F2E52427421FBFCC6825F00C0524F009
:1037D00004042543092E0CD80124B44040F2E52608
:1037E00034421FBF28F44074D1E90567344344EAEA
:1037F00007084FF68C74CFF6FE740EEA040747EA0A
:103800000C07C3F804809F614F6809695F631D62FC
:103810009F6947F008079F619F6927F004079F6130
:1038200092E100BF036842F600461D6A1A6AC4F2BC
:10383000010622F010021A621A465C6852F818EF6C
:10384000B3428E68D1F800C025F0200545EA061580
:103850000BD045F20006C4F20106B34205D043F294
:103860000046C4F20106B34207D1CE686FF04007AC
:1038700025F0C00507EA06163543A3F18046A6F5F4
:1038800096364FEAB626092E0ED8012707FA06F615
:1038900040F2E5273E421FBF24F44064D1E90567AA
:1038A00044EA860444EA870448F6FF46CFF6FF66FA
:1038B0000EEA060747EA0C275C609F614F680969BA
:1038C0009F631D629F6947F400679F619F6927F4AA
:1038D00080679F6137E100BF036842F600461D6ABA
:1038E0001A6AC4F2010622F480721A621A465C68EF
:1038F00052F81CCFB3428E68D1F800E025F4007571
:1039000045EA06250BD045F20006C4F20106B34293
:1039100005D043F20046C4F20106B34207D1CE6897
:1039200040F2FF47360225F44065BE433543A3F11C
:103930008046A6F596364FEAB626092E0ED8012700
:1039400007FA06F640F2E5273E421FBF24F4405432
:10395000D1E9056744EA061444EA07144FF68C7669
:10396000CFF6FE760CEA060747EA0E075C60DF61D9
:103970004F680969DF631D62DF6947F00807DF618F
:10398000DF6927F00407DF61DEE000BF036842F66D
:1039900000461D6A1A6AC4F2010622F480521A62B5
:1039A0001A465C6852F81CCFB3428E68D1F800E02A
:1039B00025F4005545EA06350BD045F20006C4F261
:1039C0000106B34205D043F20046C4F20106B342F9
:1039D00007D1CE6844F6FF77360325F44045BE4351
:1039E0003543A3F18046A6F596364FEAB626092E52
:1039F0000ED8012707FA06F640F2E5273E421FBF20
:103A000024F44044D1E9056744EA861444EA871463
:103A100048F6FF46CFF6FF660CEA060747EA0E2790
:103A20005C60DF614F6809691F641D62DF6947F4EC
:103A30000067DF61DF6927F48067DF6183E000BF33
:103A40000368D3F820C01A6AA3F1804722F48032B9
:103A50001A621A46A7F596375D6852F8508FD1F86A
:103A600000E08E684FEAB727092F0AD80124BC402E
:103A700040F2E5273C421EBF4C6925F4803545EAFB
:103A800004252CF4003747EA06474FF68C76CFF62C
:103A9000FE76033606EA080646EA0E065D601E65F7
:103AA0004E6809699E641F621F6D47F008071F6515
:103AB0001F6D27F004071F6546E000BF01210022AB
:103AC00080F83C200846BDE8F08100BF0368D3F8C9
:103AD00020C01A6AA3F1804722F480121A621A46A3
:103AE000A7F596375D6852F8508FD1F800E08E68E0
:103AF0004FEAB727092F0AD80124BC4040F2E52736
:103B00003C421EBF4C6925F4802545EA84252CF4EF
:103B1000001747EA065748F6FF46CFF6FF6606F558
:103B2000407606EA080646EA0E265D601E654E6887
:103B30000969DE641F621F6D47F400671F651F6D12
:103B400027F480671F65090213681943116000217B
:103B5000002280F83C200846BDE8F081002804BF20
:103B60000120704710B5044690F83D0028B90020A8
:103B700084F83C00204600F023F8022084F83D0041
:103B80002068211D01F02CF9012084F8480084F8F8
:103B90003E0084F83F0084F8400084F8410084F837
:103BA000420084F8430084F8440084F8450084F817
:103BB000460084F8470084F83D00002010BD000056
:103BC0007047000061B10A1F4FEAB202032A15D8FC
:103BD000DFE802F00218101C00F13F0318E000BFFC
:103BE00090F83E20012A1CBF01207047022280F875
:103BF0003E202CE000F141030AE000BF00F1430346
:103C000006E000BF00F1400302E000BF00F1420304
:103C10001B78012B1CBF01207047032A0CD8DFE85A
:103C200002F0030F071300BF022280F83F200EE0CE
:103C3000022280F841200AE0022280F8432006E0B8
:103C4000022280F8402002E0022280F8422002682E
:103C500001F01F010120136A00FA01F18B43136286
:103C6000136A0B43A2F18041A1F596314FEAB121CD
:103C70000729136258D8884010F0E50F54D0506CD3
:103C800042F6FF31C4F2010140F400408A42506420
:103C90000EDC40F2FF70C4F20000824218DCB2F188
:103CA000804F2DD040F20040C4F2000026E000BF5B
:103CB00043F6FF70C4F20100824215DC42F6004078
:103CC000C4F2010082421BD043F2004014E000BF66
:103CD00040F60000C4F20000824211D040F60040DD
:103CE000C4F200000AE000BF45F20000C4F2010087
:103CF000824205D044F20000C4F2010082420CD19D
:103D000090680721C0F20101014006294FF0000030
:103D100008D0B1F5803F08BF7047106840F001003F
:103D200010600020704700BF42F6FF30C4F201006F
:103D30008242AEDD43F6FF70C4F201008242BDDD77
:103D400044F20000C4F201008242D9D045F20000E2
:103D5000C4F201008242E0D1506C40F40040506453
:103D6000CEE7000090F88410012904BF02207047BC
:103D70002421C0F8881002681168136823F0010339
:103D8000136021F000530021416613602022C0F827
:103D9000882080F88410084670470000B0B590F87D
:103DA0008420012A04BF0220B0BD2422C0F888204C
:103DB0000268D0F864E0D2F800C01368BEF1000FCA
:103DC00023F001031360936823F0606341EA030169
:103DD000916019D09368916846F6A00E490FC0F61D
:103DE000000E46F6A8051EF80140C0F60005695C05
:103DF000C3F34263E400B4FBF1F11EF80340EB5C53
:103E0000E500B5FBF3F301E001210123A0F86A10FE
:103E10002021A0F86830C2F800C0C0F88810002146
:103E200080F884100846B0BDB0B590F88420012A0F
:103E300004BF0220B0BD2422C0F888200268D0F858
:103E400064E0D2F800C01368BEF1000F23F0010354
:103E50001360936823F0604341EA0301916019D035
:103E60009368916846F6A00E490FC0F6000E46F61C
:103E7000A8051EF80140C0F60005695CC3F3426363
:103E8000E400B4FBF1F11EF80340EB5CE500B5FB88
:103E9000F3F301E001210123A0F86A102021A0F82A
:103EA0006830C2F800C0C0F88810002180F8841083
:103EB0000846B0BD10B5D8B10446D0F8880028B97E
:103EC000002084F88400204600F026F82420C4F85E
:103ED00088002068A16A026822F00102026011B124
:103EE000204601F02FF8204601F058F9012801D1B1
:103EF000012010BD2168486820F49040486088681F
:103F000020F02A008860086840F0010220460A601C
:103F1000BDE8104001F08AB870B59CB0044600209E
:103F20001B90CDE91900CDE9170002A85421FCF738
:103F3000A7F9206844F60001C4F20001884239D094
:103F400043F60001C4F20101884265D048F2000145
:103F5000C4F2000188425DD12020029002A8FEF741
:103F600057F9002818BFFCF7CBFD41F24C00C4F212
:103F70000200016941F001010161016901F00101E3
:103F800001910199016841F001010160006802217D
:103F900000F00100019001980C2018910021179069
:103FA000CDE919111B9017A94FF09040FDF7D0FDF6
:103FB0001CB070BD0420029002A8FEF729F9002869
:103FC00018BFFCF79DFD41F24C00C4F20200C1682D
:103FD00041F48021C160C16801F4802101910199FF
:103FE000016841F002010160006817A900F00200B9
:103FF000019001984FF42060179002201890002043
:10400000CDE9190007201B9040F20040C4F60000E3
:10401000FDF79EFD1CB070BD0120029002A8FEF7C6
:10402000F7F8002818BFFCF76BFD41F24C00C4F212
:1040300002004169002641F480414161416901F477
:10404000804101910199016841F00401016000681B
:1040500017A900F004000190019830201790022069
:10406000189007201B9040F20040C4F6000000F5B5
:104070008060CDE91966FDF76BFD40F2D035442034
:10408000C2F20005C4F202001921102285E847009F
:104090004FF4805080234FF0200C28622846C5E959
:1040A0000436C5E9066CFDF7E7FA002818BFFCF7EF
:1040B00027FDE567AC621CB070BD0000FEE70000A4
:1040C00040F69000C2F2000090ED001A9FED062A23
:1040D0009FED063A20EE020A21EE031A31EE000AA5
:1040E00080ED000A704700BFCDCCCC3D6666663FD0
:1040F00010B58CB040F26C10C2F200004FF0A0413D
:1041000000244FF4403201234FF0040C80E81600E5
:1041100003210B94CDE90944CDE90744CDE90544D9
:10412000CDE90344CDE90144C0E90344C0E9053CBD
:104130008483016280F82430C0E90A34046380F883
:104140003840C46380F84040FCF7D8FF002818BF0F
:10415000FCF7D6FC40F26C10C2F2000009A90994E9
:10416000FCF73EFD002818BFFCF7CAFC0220C0F295
:104170003040019006207F2102900020049104210C
:104180000390CDE9051040F26C10C2F2000001A9C5
:10419000FCF7C0FD002818BFFCF7B2FC0420C0F6F5
:1041A000600001900C20029040F26C10C2F20000FE
:1041B00001A9FCF7AFFD002818BFFCF7A1FC40F2F5
:1041C0000020C2F2B05001901220029040F26C1018
:1041D000C2F2000001A9FCF79DFD002818BFFCF702
:1041E0008FFC0CB010BD0000B0B588B040F2D81004
:1041F00040F20011C2F20000C5F2000100244FF4A9
:1042000040320123042580E816000321CDE906444D
:10421000CDE90444CDE90244CDE90044C0E90344BA
:10422000C0E905358483016280F82430C0E90A348E
:10423000046380F83840C46380F84040FCF75EFFB8
:10424000002818BFFCF75CFC0820C0F690400090E6
:104250000620CDE901047F20CDE9030540F2D81006
:10426000C2F2000069460594FCF754FD002818BF0F
:10427000FCF746FC1020C1F2C00000900C20019019
:1042800040F2D810C2F200006946FCF743FD002856
:1042900018BFFCF735FC41F20000C3F2602000902B
:1042A0001220019040F2D810C2F200006946FCF7DB
:1042B00031FD002818BFFCF723FC08B0B0BD00009A
:1042C00010B58CB040F2442040F20041C2F2000030
:1042D000C5F2000100244FF4403280E816004FF48C
:1042E0008071042381830121CDE90A44CDE907448B
:1042F000CDE90544CDE90344CDE90144C0E90344D7
:10430000C0E90543016280F82440C0E90B4480F80D
:104310003840C46380F84040FCF7F0FE002818BF26
:10432000FCF7EEFB40F24420C2F2000009A9099418
:10433000FCF756FC002818BFFCF7E2FB0220C0F295
:104340003040019006207F2102900020049104213A
:104350000390CDE9051040F24420C2F2000001A90B
:10436000FCF7D8FC002818BFFCF7CAFB0CB010BD46
:1043700080B582B041F24800C4F202000168002218
:1043800041F004010160016801F00401019101990B
:10439000016841F0010101600068002100F00100A6
:1043A000009000980B20FDF759FE0B20FDF746FE0C
:1043B0000C2000210022FDF751FE0C20FDF73EFEEF
:1043C0000D2000210022FDF749FE0D20FDF736FEED
:1043D0000E2000210022FDF741FE0E2002B0BDE8B4
:1043E0008040FDF72BBE000080B540F2304046F221
:1043F0000041C2F20000C4F200010022C0E9001234
:104400004FF0100C01230221C0E90222C0F80F2056
:10441000C0E905C3C0E90711C0E90933C0E90B339E
:10442000C0E90D22C263FDF7D1F9002808BF80BDA5
:10443000BDE88040FCF764BB80B540F2944046F68E
:104440000001C2F20000C4F200010022C0E9001223
:104450004FF0100C01230221C0E90222C0F80F2006
:10446000C0E905C3C0E90711C0E90933C0E90B334E
:10447000C0E90D22C263FDF7A9F9002808BF80BD7D
:10448000BDE88040FCF73CBB2DE9F04186B000263A
:1044900041F24C00CDE90466C4F20200016840F626
:1044A000000441F0040101600168C4F6000401F059
:1044B0000401009100990168002241F0200101608F
:1044C00001684FF4007701F0200100910099016824
:1044D00041F001010160016801F0010100910099C2
:1044E000016841F002010160016801F002010091E0
:1044F0000099016841F00801016000684FF4007103
:1045000000F00800009000982046FDF70FFC4FF0E7
:1045100090404FF4806100224FF48068FDF706FC64
:104520004FF4005001904FF4881001ADCDE9020620
:1045300020462946FDF70CFB019701272046294616
:10454000CDE902760496FDF703FB4FF09040294633
:10455000CDE90187CDE90366FDF7FAFA28200021AD
:104560000022FDF77BFD2820FDF768FD06B0BDE8C1
:10457000F081000080B540F2F84045F20041C2F2FF
:104580000000C4F2000142F272120023C0F2800265
:104590004FF0010C80E80E10C0E90433C0E9063387
:1045A0000362FDF719FC002818BFFCF7A9FA40F2D6
:1045B000F840C2F200000021FDF7C4FB002818BF3C
:1045C000FCF79EFA40F2F840C2F200000021FDF72D
:1045D000DFFB002818BFFCF793FA0420C4F20100A7
:1045E000016841F48011016080BD000080B540F297
:1045F0004C5045F60001C2F20000C4F2000142F244
:1046000072120023C0F280024FF0010C80E80E10FD
:10461000C0E90433C0E906330362FDF7DDFB00287F
:1046200018BFFCF76DFA40F24C50C2F200000021B6
:10463000FDF788FB002818BFFCF762FA40F24C50E7
:10464000C2F200000021FDF7A3FB002818BFFCF711
:1046500057FA0420C4F20100016841F4001101601E
:1046600080BD000080B540F2A05048F20001C2F2C7
:104670000000C4F2000143F2243200234FF00C0C7E
:10468000C0F2030280E80E00C0E90333C0E905C3AD
:10469000C0E908338362FFF70DFC002818BFFCF760
:1046A0002FFA40F2A050C2F200000021FFF7BCFB3D
:1046B000002818BFFCF724FA40F2A050C2F2000014
:1046C0000021FFF76BFB002818BFFCF719FA40F236
:1046D000A050C2F20000FFF745FB002808BF80BDD4
:1046E000BDE88040FCF70CBA10B59CB0002401A8CE
:1046F00034211B94CDE91944CDE91644CDE9144485
:10470000CDE91244CDE91044CDE90E44FBF7B8FDE4
:1047100040F2346042F60041C2F20000C4F20101EE
:1047200041F27B52C0E90014C0E90242C0E90444EE
:104730008461FEF7CDFC002818BFFCF7E1F94FF4C7
:104740008050189040F23460C2F2000018A9FEF7C1
:104750001FFD002818BFFCF7D3F940F23460C2F205
:104760000000FFF7FBF9002818BFFCF7C9F940F279
:1047700034600024C2F2000015A9CDE91544179455
:10478000FEF7ACFB002818BFFCF7BAF96020CDE9B2
:104790000E0440F23460C2F200000EA90022CDE9FE
:1047A0001044CDE912441494FEF7D8FF002818BF36
:1047B000FCF7A6F94FF4FA700F9040F23460C2F2A1
:1047C00000000EA90422FEF7C9FF002818BFFCF75D
:1047D00097F940F23460C2F200000EA90822FEF7F9
:1047E000BDFF002818BFFCF78BF900204FF40051E3
:1047F000CDE906104FF000710590CDE90300CDE939
:104800000100CDE90800CDE90A10CDE90C0040F225
:104810003460C2F2000001A9FEF7C6FA002818BFF2
:10482000FCF76EF940F23464C2F200042046002125
:10483000FFF7C8F920460421FFF7C4F920460821F4
:10484000FFF7C0F920460021FEF7B8FB20460421FF
:10485000FEF7B4FB20460821FEF7B0FB2046FEF72A
:104860000DFF1CB010BD000010B592B040F280608A
:104870000024C2F200004FF08041C0E9001403217F
:10488000CDE90914012140F6FF72CDE90B14CDE901
:104890000F1409A90894CDE90644CDE90444CDE9F3
:1048A0000244CDE90044C0E9024204618461CDE9DB
:1048B0000D441194FEF77CFD002818BFFCF720F989
:1048C00040F28060C2F2000006A906940894FEF748
:1048D00005FB002818BFFCF713F90020CDE9040000
:1048E000CDE9000002908DF80C0040F28060C2F229
:1048F00000006946FEF7C2FA002818BFFCF700F96D
:1049000012B010BD10B592B040F2CC6040F2004140
:104910000024C2F20000C4F20001C0E90014032127
:10492000CDE90914012140F6FF72CDE90B14CDE960
:104930000F1409A90894CDE90644CDE90444CDE952
:104940000244CDE90044C0E9024204618461CDE93A
:104950000D441194FEF72CFD002818BFFCF7D0F889
:1049600040F2CC60C2F2000006A906940894FEF75B
:10497000B5FA002818BFFCF7C3F80020CDE9040001
:10498000CDE9000002908DF80C0040F2CC60C2F23C
:1049900000006946FEF772FA002818BFFCF7B0F86D
:1049A00012B010BD10B59CB0002401A834211B9496
:1049B000CDE91944CDE91644CDE91444CDE91244BA
:1049C000CDE91044CDE90E44FBF75AFC40F21870D3
:1049D00043F20041C2F20000C4F2010141F27B52F5
:1049E000C0E90014C0E90242C0E904448461FEF752
:1049F0006FFB002818BFFCF783F84FF48050189025
:104A000040F21870C2F2000018A9FEF7C1FB00289E
:104A100018BFFCF775F840F21870C2F20000FFF7FB
:104A20009DF8002818BFFCF76BF840F218700024BE
:104A3000C2F2000015A9CDE915441794FEF74EFA0D
:104A4000002818BFFCF75CF860200E904FF4FA7055
:104A5000CDE90F0440F21870C2F200000EA9002246
:104A6000CDE91144CDE91344FEF778FE002818BFC4
:104A7000FCF746F840F21870C2F200000EA90422BA
:104A8000FEF76CFE002818BFFCF73AF840F21870E9
:104A9000C2F200000EA90822FEF760FE002818BF2F
:104AA000FCF72EF800204FF40051CDE906104FF02E
:104AB00000710590CDE90300CDE90100CDE90800C2
:104AC000CDE90A10CDE90C0040F21870C2F20000E6
:104AD00001A9FEF769F9002818BFFCF711F840F2A8
:104AE0001870C2F20000FEF7C9FD1CB010BD000036
:104AF00080B540F2647043F60001C2F20000C4F2D7
:104B0000010100234FF00C0C4FF4E12280E80E006D
:104B1000C0E90333C0E905C3C0E90733C0E909337D
:104B2000FFF7C8F9002818BFFBF7EAFF40F26470EE
:104B3000C2F200000021FFF777F9002818BFFBF749
:104B4000DFFF40F26470C2F200000021FFF726F997
:104B5000002818BFFBF7D4FF40F26470C2F20000D7
:104B6000FFF700F9002808BF80BDBDE88040FBF7D3
:104B7000C7BF000080B540F2F87044F60001C2F2F1
:104B80000000C4F2000100234FF00C0C4FF4E1329E
:104B900080E80E00C0E90333C0E905C3C0E907336C
:104BA000C0E90933FFF786F9002818BFFBF7A8FF13
:104BB00040F2F870C2F200000021FFF735F900283A
:104BC00018BFFBF79DFF40F2F870C2F20000002111
:104BD000FFF7E4F8002818BFFBF792FF40F2F870E7
:104BE000C2F20000FFF7BEF8002808BF80BDBDE894
:104BF0008040FBF785BF0000FEE7000040F2200088
:104C0000C2F2000090ED001AB1EE080AB4EE401AAC
:104C1000F1EE10FA02DD80ED000A08E0B9EE080AB4
:104C2000B4EE401AF1EE10FAB8BF80ED000A90ED34
:104C3000011AB1EE080AB4EE401AF1EE10FA03DDE3
:104C400080ED010A09E000BFB9EE080AB4EE401A8F
:104C5000F1EE10FAB8BF80ED010A90ED021AB1EE44
:104C6000080AB4EE401AF1EE10FA03DD80ED020AF4
:104C7000704700BFB9EE080AB4EE401AF1EE10FA20
:104C8000B8BF80ED020A7047FEE7000040F22C003A
:104C90004CF6CD42C2F20000C3F64C5241F26F23F3
:104CA000026141F26F22C3F603234FF07A5CC3F630
:104CB00003324361C0F818C04CF2AC5C42638363BA
:104CC00045F2EC124DF20A730021C3F2277CC3F6C1
:104CD0003852C3F6A333C0E90011C0E90211C16123
:104CE000C0E90811C0E90A110163C0F83CC0C0E97D
:104CF0001011C0E91211C0E91411C0E91623C0E96E
:104D0000181181667047000070470000704700006E
:104D100040F25000C2F20000B0EE401A90ED080AD6
:104D200090ED032A90ED043A90ED054A30EE010A29
:104D300090ED065A20EE044A23EE013A31EE422A63
:104D400033EE043A25EE022A32EE032A9FED0E3AA4
:104D50009FED0E4AB4EE430A80ED021ABDEEC22A60
:104D6000F1EE10FAB8BFB0EE430AB4EE440AF1EE29
:104D700010FAB8BFB0EE404AB8EEC20A80ED084A59
:104D800080ED031A704700BF00803BC500803B45A3
:104D9000FDF7F6B84EF68850CEF20000016841F4F7
:104DA000700101607047000010B540F28064C2F2EB
:104DB000000420463C21FEF703FC2046BDE81040DD
:104DC000FEF784B810B540F2CC64C2F2000420466D
:104DD0003C21FEF7F5FB2046BDE81040FEF776B813
:104DE00080B540F6FF330268C4F2000343F2FF3C93
:104DF0009842C4F2010C0BDD60452FDC40F6004305
:104E0000C4F20003984235D042F600432EE000BFC2
:104E1000B0F1804F2ED040F20043C4F2000398421C
:104E200028D040F60003C4F20003984222D0604527
:104E300026DC40F2FF73C4F20003984236DD40F6F0
:104E40000003C4F20003984244D040F60043C4F289
:104E5000000398423ED042F6004337E045F200039B
:104E6000C4F20103984205D043F20043C4F20103A7
:104E70009842DCD14B6822F070021A436045D8DDBD
:104E800044F2FF33C4F20103984217DD44F20043B9
:104E9000C4F2010398421DD045F20003C4F201039D
:104EA000984217D044F6000310E000BFB0F1804FE5
:104EB00010D040F20043C4F2000309E043F2004383
:104EC000C4F20103984205D044F20003C4F2010386
:104ED000984203D1CB6822F440721A434B6922F006
:104EE000800E8A6843EA0E03D1F800C00360C262F4
:104EF000A0F18042A2F596324FEAB222092AC0F808
:104F000028C008D8012303FA02F240F2E5231A422E
:104F10001CBF09690163012141610169C90708BF1B
:104F200080BD016921F00101016180BDD0F808C098
:104F300011432CF47F4C41EA032141EA0C018160CA
:104F40007047000080B5816A0A070DD4CA0716D1E0
:104F50008A071FD44A0728D4CA0631D48A063AD40D
:104F60004A0658D542E000BF0268D0F838C05368FE
:104F700023F4004343EA0C035360CA07E8D00268F5
:104F8000D0F82CC0536823F4003343EA0C03536079
:104F90008A07DFD50268D0F830C0536823F4803325
:104FA00043EA0C0353604A07D6D50268D0F834C0F0
:104FB000536823F4802343EA0C035360CA06CDD51B
:104FC0000268D0F83CC0936823F4805343EA0C0392
:104FD00093608A06C4D50268D0F840C0936823F471
:104FE000005343EA0C0393604A0614D50268D0F8D4
:104FF00044C05368BCF5801F23F4801343EA0C03BC
:10500000536008D1D2F804C0D0F848E02CF4C003B3
:1050100043EA0E035360090658BF80BD0168C06CA7
:105020004A6822F400221043486080BDB0B582B0C7
:1050300004460020C4F89000FCF77EFE2168054677
:105040000A68120737D56FF07E4C20464FF40011E6
:1050500000222B46CDF800C000F000FA50B300BF8C
:10506000206850E8000F216820F0800041E800022D
:10507000DAB1206850E8000F216820F0800041E894
:10508000000292B1206850E8000F216820F08000F3
:1050900041E800024AB1206850E8000F216820F082
:1050A000800041E80002002ADAD12020C4F88800FC
:1050B00060E000BF21680868400761D56FF07E4C52
:1050C00020464FF4800100222B46CDF800C000F0AE
:1050D000C5F9002854D000BF206850E8000F2168AF
:1050E00020F4907041E80002E2B1206850E8000F1F
:1050F000216820F4907041E800029AB1206850E8DD
:10510000000F216820F4907041E8000252B120683D
:1051100050E8000F216820F4907041E80002002A56
:10512000DAD100BF206850E8020F216820F00100AA
:1051300041E80202DAB1206850E8020F216820F04D
:10514000010041E8020292B1206850E8020F216894
:1051500020F0010041E802024AB1206850E8020F45
:10516000216820F0010041E80202002ADAD1202063
:10517000C4F88C000320002184F8841002B0B0BD74
:105180002020C4F88800C4F88C000020E066206766
:10519000002184F8841002B0B0BD000070B5044650
:1051A0002269D4E9021300680A436169E669114380
:1051B000026846F6F315CCF6FF7531432A401143D9
:1051C0000160416848F2000C21F4405119434160EC
:1051D000A269C4F2000C60451CBF216A0A438168C1
:1051E0004FF2FF43C1F2FF13194011438160C16ABE
:1051F000D4F824E021F00F0141EA0E01C16244F627
:10520000FF71C4F2000188424FF0100318DC44F231
:105210000041C4F20001884228D044F60001C4F2E3
:10522000000188422AD044F60041C4F200018842BD
:1052300042D141F28801C4F2020109688B0933E0CE
:1052400045F20001C4F2000188421FD0604525D01C
:1052500043F60001C4F2010188422DD141F28801D8
:10526000C4F202010B6879A222E000BF41F288017A
:10527000C4F2020109688B0816E000BF41F2880100
:10528000C4F2020109680B090EE000BF41F2880177
:10529000C4F2020109680B0A06E000BF41F288016E
:1052A000C4F2020109688B0A46F69002C0F60002B9
:1052B00003F0030152F82130604542F20040C0F291
:1052C000F40015D0B6F5004F24D1082B4FF00101A2
:1052D00000F2B380DFE803F0065E6CB164B1B1B1F7
:1052E0006A0000BFFDF78AFA002856D15CE000BFD3
:1052F000082B4FF0010100F2A080DFE803F0059ECB
:10530000259E1D9E9E9E2300FDF778FAC0B1D4F81D
:1053100024E019E0082B4FF0010100F28E80DFE855
:1053200003F00565738C6B8C8C8C7100FDF766FA4D
:1053300000285ED164E000BFFDF78CFA0028E6D1BA
:1053400000217AE04FF4004046F67801C0F60001F3
:1053500031F81E106268B0FBF1F002EB42018842A6
:105360004FF0010169D31303984266D8010E000281
:1053700010EB520041F100010023FAF749FF4FF60C
:105380000052A0F54071C0F20F0291424FD30121AB
:1053900053E000BFFDF748FA30B1D4F824E007E04D
:1053A000FDF758FA0028F8D1002146E04FF40040FC
:1053B00046F67801C0F6000131F81E106268B0FBB5
:1053C000F1F0510801EB4000B0FBF2F04FF6EF7244
:1053D000A0F11001914207D84FF6F0710140C0F3DF
:1053E0004200084423E000BF012126E0FDF71CFA3B
:1053F00030B1D4F824E007E0FDF72CFA0028F8D10A
:1054000000211AE04FF4004046F67801C0F6000192
:1054100031F81E104FF6EF72B0FBF1F0616800EB4F
:105420005100B0FBF1F0A0F11001914204D82168C5
:10543000C860002101E000BF01214FF00110A0660B
:10544000002208466267A26770BD00BF010000002D
:105450000400000002000000080000002DE9F041F7
:10546000804600681546C2690E461140891BB1FA94
:1054700081F14909A94223D1069C2CB3611C29D191
:10548000C1693140891BB1FA81F14909A94217D19B
:10549000C1693140891BB1FA81F14909A9420FD193
:1054A000C1693140891BB1FA81F14909A94207D18B
:1054B000C1693140891BB1FA81F14909A942DFD0A4
:1054C0000020BDE8F08100BFFCF736FC0320BDE8FA
:1054D000F08100BF1F4607E0C0693040801BB0FA72
:1054E00080F04009A842EBD1FCF726FCC01BA0428B
:1054F00042D8D8F8000001684907EDD5402EEBD01E
:10550000802EE9D0C16909073AD4C1690905E3D5FC
:105510004FF40061016250E8000FD8F8001020F449
:10552000907041E80002002A60D0D8F8000050E8EE
:10553000000FD8F8001020F4907041E80002002A13
:1055400054D0D8F8000050E8000FD8F8001020F42C
:10555000907041E80002002A48D0D8F8000050E8D6
:10556000000FD8F8001020F4907041E80002EAB370
:10557000D8F80000CFE700BF0320BDE8F08100BFEE
:105580000821016250E8000FD8F8001020F4907054
:1055900041E80002002A00F09780D8F8000050E8A7
:1055A000000FD8F8001020F4907041E80002002AA3
:1055B00000F08A80D8F8000050E8000FD8F80010FA
:1055C00020F4907041E80002002A7DD0D8F8000055
:1055D00050E8000FD8F8001020F4907041E8000265
:1055E000002A71D0D8F80000CCE700BF4FF6FE705B
:1055F000CEF6FF70D8F8001051E8021FD8F800204E
:10560000014042E80213F3B1D8F8001051E8021F3C
:10561000D8F80020014042E80213A3B1D8F80010E6
:1056200051E8021FD8F80020014042E8021353B1AC
:10563000D8F8001051E8021FD8F80020014042E8D5
:105640000213002BD6D1D8F86C0001282CD1D8F841
:10565000000050E8000FD8F8001020F0100041E8DA
:1056600000020AB3D8F8000050E8000FD8F8001084
:1056700020F0100041E80002B2B1D8F8000050E874
:10568000000FD8F8001020F0100041E800025AB1D5
:10569000D8F8000050E8000FD8F8001020F01000F3
:1056A00041E80002002AD2D120200021C8F88C0055
:1056B000C8F86C10C8F87410C8F89000032088F877
:1056C0008410BDE8F08100BF4FF6FE70CEF6FF708B
:1056D000D8F8001051E8021FD8F80020014042E835
:1056E0000213F3B1D8F8001051E8021FD8F80020D7
:1056F000014042E80213A3B1D8F8001051E8021F9C
:10570000D8F80020014042E8021353B1D8F8001045
:1057100051E8021FD8F80020014042E80213002B94
:10572000D6D1D8F86C0001282CD1D8F8000050E868
:10573000000FD8F8001020F0100041E800020AB372
:10574000D8F8000050E8000FD8F8001020F0100042
:1057500041E80002B2B1D8F8000050E8000FD8F8D4
:10576000001020F0100041E800025AB1D8F8000003
:1057700050E8000FD8F8001020F0100041E80002B7
:10578000002AD2D12020C8F88C0000200821C8F8B7
:105790006C00C8F87400C8F8901088F884000120E4
:1057A000BDE8F081FEE7000094B0FCF7F7FB0024B1
:1057B0000020CDE90B44CDE90944CDE90744FCF7CD
:1057C00089FC4FF48071099140210A910421022043
:1057D0000F9155210690CDE90D00CDE91010CDE9CE
:1057E000120006A8FDF774F820B1EFF3108072B62E
:1057F000FEE700BF0F2001900320CDE9020401A8BD
:105800000421CDE90444FCF76FFE28B1EFF31080CA
:1058100072B600BFFEE700BFFEF736FEFEF7A8FD3A
:10582000FEF720FFFFF764F9FEF75EFFFFF7BAF817
:10583000FEF75EFCFEF7D8FCFEF79CFEFEF7D6FEF8
:10584000FFF798F9FEF7D0FDFEF73AFDFEF7F4FDFD
:10585000FFF70AF8FFF756F840F20C10C2F200000A
:10586000FBF724F940F22810C2F20000FBF71EF902
:1058700040F24410C2F20000FBF718F940F20404B1
:10588000C2F2000494ED020AFBF7A2F9D4E9000188
:10589000FBF73EF9FFF788FAFFF794FA4FF09040D4
:1058A0004FF480610122FCF741FA40F60000C4F693
:1058B00000004FF400710122FCF738FA9FED038AD3
:1058C000B0EE480AFBF790F8FAE700BF0000C842C4
:1058D0002DE9F04F81B02DED088B82B040F20C071E
:1058E000C2F2000797ED001ABEEE002A21EE028AEE
:1058F000B4EE408AF1EE10FA0CDCB6EE002A21EE8E
:10590000021AB4EE401AF1EE10FAB8BFB0EE410A36
:10591000B0EE408A10EE900AFAF745FE41EC100B0B
:105920009FEDAB1B00F0E8F951EC100BFAF74EFEBF
:105930009FEDAF0A01EE100A18EE104A31EE009A00
:10594000B5EE401A84F00040F1EE10FAA8BFB0EEB8
:10595000419AFAF728FE054619EE100A0E46FAF7A4
:1059600022FE41EC180BB0EE480AF0EE680A00F097
:1059700047FA51EC100B2A463346FAF733FDFAF793
:1059800025FE40F2FC06C2F2000630602046FAF71F
:105990000AFEB0EE480AF0EE680A04460D4600F032
:1059A00047F951EC100B22462B46FAF71BFDFAF78C
:1059B0000DFE40F2041197ED008AC2F2000196ED4F
:1059C00000AAB6EE000A086028EE00BA40F2F8011C
:1059D0003AEE0B9AC2F2000181ED009AFAF7E3FD6C
:1059E00082461AEE100A8B46FAF7DDFD9FED7A0B20
:1059F000044601900D46009153EC102B5046594639
:105A0000FAF7F0FC22462B46FAF7E6FC9FED740B02
:105A100054EC105B2A462346FAF7E4FC80461BEE62
:105A2000100A8946FAF7BFFD42464B4606460F4626
:105A3000FAF731FCFAF7CAFD40F200119FED6A0B4C
:105A4000C2F200010AEE100A086053EC102B504617
:105A50005946FAF7C7FCDDE90032FAF7BDFC2A46E1
:105A60002346FAF7BFFC02460B4630463946FAF7A2
:105A700012FCFAF7ABFD40F20811C2F200019FEDF3
:105A80005D0A0860B5EE409A40F21C01F1EE10FA92
:105A9000C2F20001B0EE401A0ADB91ED001AB4EE3A
:105AA000491AF1EE10FAB8BFB0EE419AB0EE491AB9
:105AB000B5EE40AA04EE100AF1EE10FAB0EE402A5C
:105AC0000ADB91ED002AB4EE4A2AF1EE10FAB8BFD3
:105AD000B0EE42AAB0EE4A2AB5EE404AF1EE10FA14
:105AE000B0EE403A0ADB91ED003AB4EE443AF1EE02
:105AF00010FAB8BFB0EE434AB0EE443A81EE081A4D
:105B000082EE082A83EE083AB7EE004A40F26010AF
:105B1000B0EE405AC2F20000B4EE441AF1EE10FAB0
:105B2000C8BFB0EE441AB5EE401AF1EE10FAC8BF85
:105B3000B0EE415A80ED005AB4EE442A40F26410AF
:105B4000F1EE10FAC8BFB0EE442AB5EE402AB0EE2E
:105B5000401AC2F20000F1EE10FAC8BFB0EE421ACD
:105B600080ED001AB4EE443A40F26810F1EE10FAFB
:105B7000C8BFB0EE443AB5EE403AC2F20000F1EED2
:105B800010FAC8BFB0EE430A9FED1B2A80ED000A51
:105B900040F23460C2F2000025EE023A006821EEC5
:105BA000021A20EE020ABCEEC33ABCEEC11ABCEEE9
:105BB000C00A80ED0D3A80ED0E1A80ED0F0A02B09A
:105BC000BDEC088B01B0BDE8F08F00BF00BF00BF87
:105BD00000000060FB211940AA4C58E87AB6FB3F50
:105BE000000000000000E03FAA4C58E87AB6FBBF76
:105BF000DB0FC9400000000000E0AB4503B4019892
:105C00004100009850EAC12018BF04204A0D18BF77
:105C100040F0010040F2FF72B2EB515F08BF40F06C
:105C20000200012808BF052002B0704700000000F4
:105C300010B52F499FED2C1B2DED020B84B005985C
:105C400020F000408842D8BF9DED040B2DDD29498E
:105C5000884209D1049840B94FF0010000F058FD86
:105C600000F026FD06B010BD05DB9DED040B00F035
:105C700013FD06B010BD68469DED040B00F024F93D
:105C800010F0030004BF9DED021B9DED000B0CD036
:105C900001280ED09DED021B9DED000B022817D0B0
:105CA000012000F061FC06B010BD00F029FB06B039
:105CB00010BD9DED021B9DED000B012000F054FC7A
:105CC00051EC100B81F0004106B041EC100B10BDFF
:105CD00000F016FB51EC100B81F0004106B041ECD6
:105CE000100B10BD000000000000000000000000CC
:105CF000FB21E93F0000F07F10B52DED040B86B0CD
:105D00009DED060B10EE100A10EE901A8DED000BB3
:105D1000002818BF0120084320F00040C0F17F6038
:105D200000F1E040C00F21D19DED080B10EE101ADC
:105D300010EE900A8DED000B002918BF01210843D9
:105D400020F00040C0F17F6000F1E040C00F0DD1B5
:105D500029490798B1EB400F04BF0698002842D0AC
:105D60000998400004BF089800283CD09DED080B1E
:105D700053EC102B9DED060B51EC100BFAF707FDC1
:105D8000CDE902019DED020B40F2FF7110EE900A89
:105D90008DED000B31EA105021D00798039900F0E7
:105DA000004001F00041884219D09DED080B8DEDB7
:105DB000040B9DED020B8DED000B10EE900A059982
:105DC00061F31E0005909DED041B9DED020B51EC4F
:105DD000110B53EC102BFAF702FBCDE902019DEDFC
:105DE000020B0AB010BD012000F092FC0AB0BDE821
:105DF000104000F05DBC00000000E0FF000000006B
:105E000010B52F499FED2C1B2DED020B84B005988A
:105E100020F000408842DCBF00209DED040B32DD05
:105E20002849884209D1049840B94FF0010000F098
:105E30006FFC00F03DFC06B010BD05DB9DED040BD2
:105E400000F02AFC06B010BD68469DED040B00F082
:105E50003BF810F0030011D0012818D09DED021B73
:105E60009DED000B02281AD000F04AFA51EC100BFD
:105E700081F0004106B041EC100B10BD9DED021BFE
:105E80009DED000B012000F06FFB06B010BD9DEDF5
:105E9000021B9DED000B00F033FA06B010BD01208F
:105EA00000F062FB51EC100B81F0004106B041ECB8
:105EB000100B10BD000000000000000000000000FA
:105EC000FB21E93F0000F07F2DE9F14F04462DED65
:105ED000020B2DED088B8AB09FEDE70B80ED020BD6
:105EE000139EE74826F0004585420ADC9DED120B23
:105EF000002084ED000B0AB0BDEC088B03B0BDE8B8
:105F0000F08FE0489FEDE0AB9FEDE1BBA84247DD9D
:105F1000E14F9FEDE39B9FEDE48B9DED120B53EC66
:105F20001A2B51EC100B002E1CDDFAF755FA41EC40
:105F3000100BBD4208D053EC1B2B51EC100BFAF7A1
:105F40004BFAC4E900010BE053EC192B51EC100B98
:105F5000FAF742FA53EC182BFAF73EFAC4E90001BB
:105F60000120C8E7FAF797F941EC100BBD4208D0C1
:105F700053EC1B2B51EC100BFAF78DF9C4E900011F
:105F80000BE053EC192B51EC100BFAF784F953EC9E
:105F9000182BFAF780F9C4E900014FF0FF30AAE7A7
:105FA000C348A84279DB9DED120B51EC100B00F0B9
:105FB000B5FB41EC180B9FEDC00B53EC102BFAF71F
:105FC00011FA9FEDBF1B53EC112BFAF764F9FAF7A6
:105FD00051FC0746FAF730FC41EC190B53EC1A2B35
:105FE000FAF700FA53EC182BFAF7F9F941EC180B11
:105FF00053EC1B2B51EC190BFAF7F4F9DFF8C8A29C
:1060000041EC100B4FEA15580125FA4453EC102BC4
:1060100051EC180BFAF7E0F9032DC4E900013DD06B
:10602000C1F30A5005EB4511A8EB0000113981427C
:1060300034DA0AEB051BB0EE48AA9BED000BF0EE3C
:1060400068AA53EC102B51EC190BFAF7CBF941EC81
:106050001B0B51EC1A0B53EC1B2BFAF7BDF941EC5F
:10606000180B51EC1A0B53EC182BFAF7B5F953EC4B
:106070001B2BFAF7B1F99BED020B41EC1A0B53EC19
:10608000102B51EC190BFAF7ADF953EC1A2BFAF768
:10609000A3F941EC100B6D1CB8E70EE0002EA8BF71
:1060A0003846BFF628AF94ED000B51EC100B81F091
:1060B0000041C4E9000178421DE7C6F3130040F433
:1060C000801EC6F30A50A0F2F530471100F01F05FC
:1060D000C5F12000DDF848B0089000200690079038
:1060E0000520EC467949002D07EB0002794408BFF2
:1060F00051F8221009D051F8223001EB8201AB4057
:106100004A68089922FA01F11943A1FB0E26A1FB66
:106110000B131A449A4234BF0123002303EB0608F1
:106120000CEB8003D3E901A60E448E4234BF01215B
:10613000002192448A4411B1924502D903E092456C
:1061400001D2012100E00021C3E901A641444CF83D
:106150002010011EA0F10100C4DC029800F10050E3
:10616000850F0298DDE903678000DDF81480FAF7F7
:1061700063FB41EC1A0B3046FAF76FFB9FED541BA3
:1061800053EC112BFAF72EF941EC1B0B3846FAF7BA
:1061900064FB9FED511B53EC112BFAF723F941ECF3
:1061A000180B4046FAF759FB9FED4D1B53EC112B92
:1061B000FAF718F941EC190B51EC180B53EC192BA9
:1061C000FAF769F853EC1B2BFAF765F853EC1A2B26
:1061D000FAF761F8CDE90801002008909DED080B61
:1061E00053EC1A2B51EC100BFAF7F6F853EC1B2B6F
:1061F000FAF7F2F853EC182BFAF7EEF853EC192BE8
:10620000FAF7EDF89FED381B53EC112BFAF7EAF88B
:106210009FED370B41EC180B53EC102B9DED080B49
:1062200051EC100BFAF7DEF853EC182BFAF733F8B1
:106230009FED310B41EC180B53EC102B9DED080B2F
:1062400051EC100BFAF7CEF853EC182BFAF723F8B1
:1062500041EC100B139810F0004F06D06D4251EC3A
:10626000100B81F0004141EC100B284684ED000B2F
:1062700041E60000000000000000000000000000F7
:10628000FB21E93F7CD9024000004054FB21F93F4B
:106290003163621A61B4D03DFB21F93F0000000078
:1062A0000000601A61B4D03D7370032E8A19A33BBD
:1062B000FB2139410000000083C8C96D305FE43F15
:1062C000000000000000E03F5A070000A8060000A0
:1062D000000000000000103E000000000000103C24
:1062E000000000000000103A182D4454FB21F93D35
:1062F0003326A611460B113C00000054FB21F93D4A
:1063000010B52DED040B2DED088B82B0B0EE419A47
:10631000F0EE619A0B9820F000449FED4BABB4F186
:10632000795F11DA9DED0A0B51EC100BFAF7A2FA26
:10633000002801BFB0EE4A0AF0EE6A0A02B0BDECD6
:10634000088B04BF04B010BD9DED0A0B53EC102B5D
:1063500051EC100BFAF746F841EC180B3C480621BB
:10636000B0EE480AF0EE680A784400F081F853EC89
:10637000182B51EC100BFAF735F89DED0A0B41EC98
:106380001B0B53EC192B51EC100BFAF72BF841ECCB
:10639000190B53EC1B2B51EC180BFAF723F853ECA9
:1063A000192BFAF719F89FED2C0B41EC190B53EC54
:1063B000102B51EC180BFAF715F841EC100B28488C
:1063C000844210DA53EC192B51EC100BFAF704F855
:1063D00053EC1A2BFAF703F841EC100B02B0BDECAA
:1063E000088B04B010BD1F48A042BCBF9FED1E1B10
:1063F0008DED001B06DBA4F500100190002000903D
:106400009DED001B51EC100B53EC112BF9F7E4FF41
:106410009DED000B41EC180B53EC102B51EC1A0BBB
:10642000F9F7DAFF41EC1A0B53EC192B51EC180B6E
:10643000F9F7D2FF53EC1A2BF9F7D1FF41EC100B0F
:10644000CCE7000000000000000000000000F03F6A
:10645000CC03000000000000000000000000E03F4E
:106460003333D33F0000E93F000000000000D23F7B
:1064700070B504462DED028B4D1E00EBC500B0EE4D
:10648000408AF0EE608A90ED000B35F0060017D0E0
:1064900053EC182B51EC100BF9F7A4FF41EC100B47
:1064A0006D1E04EBC50090ED001B51EC100B53EC7E
:1064B000112BF9F7F0FE41EC100B35F00600E7D197
:1064C000022D36D0042D1CD0062D1CBFBDEC028B36
:1064D00070BD53EC182B51EC100BF9F783FF94EDC2
:1064E0000A1B53EC112BF9F7D6FE53EC182BF9F7D6
:1064F00079FF94ED081B53EC112BF9F7CCFE41EC1E
:10650000100B53EC182B51EC100BF9F76BFF94EDBB
:10651000061B53EC112BF9F7BEFE53EC182BF9F7C1
:1065200061FF94ED040B53EC102BF9F7B4FE41EC32
:10653000100B53EC182B51EC100BF9F753FF94EDA3
:10654000021B53EC112BF9F7A6FE53EC182BF9F7AD
:1065500049FF94ED001B53EC112BF9F79CFEBDECA9
:10656000028B41EC100B70BD31B504462DED040BD0
:106570002DED0A8BB0EE41BAF0EE61BA0B989DEDAD
:106580000A0B20F00040B0F1795F0DDA51EC100BEE
:10659000FFF734FB042808BF00F09AF89DED0A0BC2
:1065A000BDEC0A8B05B030BD53EC102B51EC100B39
:1065B000F9F718FF41EC180B9DED0A0B53EC182B63
:1065C00051EC100BF9F70EFF41EC190B2C48B0EE13
:1065D000480AF0EE680A05217844FFF749FF9FED6D
:1065E0002ACBB0EE40AAF0EE60AA9CB353EC1C2B71
:1065F00051EC190BF9F7F6FE41EC1C0B53EC1A2B7E
:1066000051EC190BF9F7EEFE9FED210B41EC190B44
:1066100053EC102B51EC1B0BF9F7E4FE53EC192B48
:10662000F9F7DAFE53EC182BF9F7DCFE53EC1B2BD1
:10663000F9F7D2FE53EC1C2BF9F7CEFE9DED0A1BA9
:1066400053EC112BF9F7CBFEBDEC0A8B05B041ECF6
:10665000100B30BDFFE753EC1A2B51EC180BF9F778
:10666000C1FE53EC1C2BF9F716FE53EC192BF9F76E
:10667000B9FE9DED0A1B53EC112BF9F70CFEE3E775
:106680005C02000000000000495555555555C5BF36
:10669000000000000000E03F10B553EC102B51EC5F
:1066A000100BF9F7F8FD41EC100B10BD00000000D5
:1066B0009FED050B10B553EC102B51EC100BF9F7B7
:1066C00003FF41EC100B10BD0000000000000000B3
:1066D0009FED050B10B553EC102B51EC100BF9F797
:1066E00081FE41EC100B10BD000000000000001006
:1066F00002E008C8121F08C1002AFAD1704770478B
:10670000002001E001C1121F002AFBD170470000E8
:1067100001490860704700000000002082B0CDE908
:10672000000121F0004001909DED000B02B051EC02
:10673000100B7047000000004C5555555555A53FAE
:106740007751C1166CC156BF9015CB19A001FA3E06
:10675000AD529C804F7E92BEC4B1B4BD9EEE213E30
:10676000D43888BEE9FAA8BD00004054FB21F93FA7
:106770003163621A61B4D03D0000601A61B4D03D4B
:106780007370032E8A19A33B0000002E8A19A33BC5
:10679000C14920259A837B390000000000000000D9
:1067A0006E83F9A22915444ED15727FCC0DD34F57C
:1067B000999562DB4190433CAB6351FE61C5BBDE02
:1067C0003A6E24B7E0D24D42EA2E49061C92D10916
:1067D0001CEB1DFE3EA729B1F53582E88444BB2E93
:1067E00026709CE9417E5FB439D69139F4395383E0
:1067F0008B5F849C3B28F9BDFF97F81F0F9805DE3F
:106800008B112FEF1F6D0A5ACF7E366DB709CB273C
:10681000663F464F2DEA5F9EC7BA27757BF1E5EBD1
:10682000F739073DEA92528AB15FFB6B085D8D1F15
:106830004630035600000000A6F810111111813FE8
:10684000D561C119A0012ABF7DFEB157E31DC73E26
:10685000EB9C2B8AE6E55ABE7CD5CF5A3AD9E53D6A
:106860000000000000000000010203040607080900
:106870000000000001020304010002000400060001
:1068800008000A000C0010002000400080000001F9
:1068900000000000040000000200000008000000EA
:1068A00001010103070100000804020408010101BD
:1068B000D06800080000002020000000F0660008FA
:1068C000F068000820000020780C00000067000835
:1068D000000000000700000001000000000040412F
:1068E00010000000010000000024F40000004041FE
:04000005080001D915
:00000001FF
